Archive member included because of file (symbol)

C:/Program Files/Microchip/MPLAB C32/bin/../lib/gcc/pic32mx/3.4.4/../../../../pic32mx/lib/size\libc.a(memcpy.o)
                              Objects - Graphics Primitives Layer Demo\MainDemo.o (memcpy)
C:/Program Files/Microchip/MPLAB C32/bin/../lib/gcc/pic32mx/3.4.4/../../../../pic32mx/lib/size\libc.a(general-exception.o)
                              C:/Program Files/Microchip/MPLAB C32/bin/../lib/gcc/pic32mx/3.4.4/../../../../pic32mx/lib/size/crt0.o (_general_exception_context)
C:/Program Files/Microchip/MPLAB C32/bin/../lib/gcc/pic32mx/3.4.4/../../../../pic32mx/lib/size\libc.a(exit.o)
                              C:/Program Files/Microchip/MPLAB C32/bin/../lib/gcc/pic32mx/3.4.4/../../../../pic32mx/lib/size/crt0.o (exit)
C:/Program Files/Microchip/MPLAB C32/bin/../lib/gcc/pic32mx/3.4.4/../../../../pic32mx/lib/size\libc.a(_iobdata.o)
                              C:/Program Files/Microchip/MPLAB C32/bin/../lib/gcc/pic32mx/3.4.4/../../../../pic32mx/lib/size\libc.a(exit.o) (_libc_data)
C:/Program Files/Microchip/MPLAB C32/bin/../lib/gcc/pic32mx/3.4.4/../../../../pic32mx/lib/size\libc.a(_iobfuncs.o)
                              C:/Program Files/Microchip/MPLAB C32/bin/../lib/gcc/pic32mx/3.4.4/../../../../pic32mx/lib/size\libc.a(_iobdata.o) (_filbuf_simple)
C:/Program Files/Microchip/MPLAB C32/bin/../lib/gcc/pic32mx/3.4.4/../../../../pic32mx/lib/size\libc.a(stubs.o)
                              C:/Program Files/Microchip/MPLAB C32/bin/../lib/gcc/pic32mx/3.4.4/../../../../pic32mx/lib/size\libc.a(exit.o) (pthread_mutex_lock)
C:/Program Files/Microchip/MPLAB C32/bin/../lib/gcc/pic32mx/3.4.4/../../../../pic32mx/lib/size\libc.a(default-general-exception-handler.o)
                              C:/Program Files/Microchip/MPLAB C32/bin/../lib/gcc/pic32mx/3.4.4/../../../../pic32mx/lib/size\libc.a(general-exception.o) (_general_exception_handler)
C:/Program Files/Microchip/MPLAB C32/bin/../lib/gcc/pic32mx/3.4.4/../../../../pic32mx/lib/size\libc.a(default-bootstrap-exception-handler.o)
                              C:/Program Files/Microchip/MPLAB C32/bin/../lib/gcc/pic32mx/3.4.4/../../../../pic32mx/lib/size/crt0.o (_bootstrap_exception_handler)
C:/Program Files/Microchip/MPLAB C32/bin/../lib/gcc/pic32mx/3.4.4/../../../../pic32mx/lib/size\libc.a(default-on-reset.o)
                              C:/Program Files/Microchip/MPLAB C32/bin/../lib/gcc/pic32mx/3.4.4/../../../../pic32mx/lib/size/crt0.o (_on_reset)
C:/Program Files/Microchip/MPLAB C32/bin/../lib/gcc/pic32mx/3.4.4/../../../../pic32mx/lib/size\libc.a(default-on-bootstrap.o)
                              C:/Program Files/Microchip/MPLAB C32/bin/../lib/gcc/pic32mx/3.4.4/../../../../pic32mx/lib/size/crt0.o (_on_bootstrap)
C:/Program Files/Microchip/MPLAB C32/bin/../lib/gcc/pic32mx/3.4.4/../../../../pic32mx/lib/size\libc.a(default-nmi-handler.o)
                              C:/Program Files/Microchip/MPLAB C32/bin/../lib/gcc/pic32mx/3.4.4/../../../../pic32mx/lib/size/crt0.o (_nmi_handler)
C:/Program Files/Microchip/MPLAB C32/bin/../lib/gcc/pic32mx/3.4.4/../../../../pic32mx/lib/size\libc.a(_mon_getc.o)
                              C:/Program Files/Microchip/MPLAB C32/bin/../lib/gcc/pic32mx/3.4.4/../../../../pic32mx/lib/size\libc.a(_iobfuncs.o) (_mon_getc)
C:/Program Files/Microchip/MPLAB C32/bin/../lib/gcc/pic32mx/3.4.4/../../../../pic32mx/lib/size\libc.a(_mon_write.o)
                              C:/Program Files/Microchip/MPLAB C32/bin/../lib/gcc/pic32mx/3.4.4/../../../../pic32mx/lib/size\libc.a(_iobfuncs.o) (_mon_write)
C:/Program Files/Microchip/MPLAB C32/bin/../lib/gcc/pic32mx/3.4.4/../../../../pic32mx/lib/size\libc.a(_exit.o)
                              C:/Program Files/Microchip/MPLAB C32/bin/../lib/gcc/pic32mx/3.4.4/../../../../pic32mx/lib/size\libc.a(exit.o) (_exit)
C:/Program Files/Microchip/MPLAB C32/bin/../lib/gcc/pic32mx/3.4.4/../../../../pic32mx/lib/size\libc.a(errno.o)
                              C:/Program Files/Microchip/MPLAB C32/bin/../lib/gcc/pic32mx/3.4.4/../../../../pic32mx/lib/size\libc.a(_iobfuncs.o) (errno)
C:/Program Files/Microchip/MPLAB C32/bin/../lib/gcc/pic32mx/3.4.4/../../../../pic32mx/lib/size\libc.a(_mon_putc.o)
                              C:/Program Files/Microchip/MPLAB C32/bin/../lib/gcc/pic32mx/3.4.4/../../../../pic32mx/lib/size\libc.a(_mon_write.o) (_mon_putc)
C:/Program Files/Microchip/MPLAB C32/bin/../lib/gcc/pic32mx/3.4.4/../../../../pic32mx/lib/size\libmchp_peripheral.a(int_disable_interrupts_lib.o)
                              Objects - Graphics Primitives Layer Demo\MainDemo.o (INTDisableInterrupts)
C:/Program Files/Microchip/MPLAB C32/bin/../lib/gcc/pic32mx/3.4.4/../../../../pic32mx/lib/size\libmchp_peripheral.a(int_enable_mv_int_lib.o)
                              Objects - Graphics Primitives Layer Demo\MainDemo.o (INTEnableSystemMultiVectoredInt)
C:/Program Files/Microchip/MPLAB C32/bin/../lib/gcc/pic32mx/3.4.4/../../../../pic32mx/lib/size\libmchp_peripheral.a(int_restore_interrupts_lib.o)
                              Objects - Graphics Primitives Layer Demo\MainDemo.o (INTRestoreInterrupts)
C:/Program Files/Microchip/MPLAB C32/bin/../lib/gcc/pic32mx/3.4.4/../../../../pic32mx/lib/size\libmchp_peripheral.a(open_core_timer_lib.o)
                              Objects - Graphics Primitives Layer Demo\DisplayDriver.o (OpenCoreTimer)
C:/Program Files/Microchip/MPLAB C32/bin/../lib/gcc/pic32mx/3.4.4/../../../../pic32mx/lib/size\libmchp_peripheral.a(pcache.o)
                              Objects - Graphics Primitives Layer Demo\MainDemo.o (CheKseg0CacheOn)
C:/Program Files/Microchip/MPLAB C32/bin/../lib/gcc/pic32mx/3.4.4/../../../../pic32mx/lib/size\libmchp_peripheral.a(int_enable_interrupts_lib.o)
                              C:/Program Files/Microchip/MPLAB C32/bin/../lib/gcc/pic32mx/3.4.4/../../../../pic32mx/lib/size\libmchp_peripheral.a(int_enable_mv_int_lib.o) (INTEnableInterrupts)

Allocating common symbols
Common symbol       size              file

_cursorY            0x2               Objects - Graphics Primitives Layer Demo\Primitive.o
_fontOrientation    0x1               Objects - Graphics Primitives Layer Demo\Primitive.o
_fontFirstChar      0x2               Objects - Graphics Primitives Layer Demo\Primitive.o
_clipRgn            0x2               Objects - Graphics Primitives Layer Demo\DisplayDriver.o
_fontHeight         0x2               Objects - Graphics Primitives Layer Demo\Primitive.o
_line_mem_pitch     0x4               Objects - Graphics Primitives Layer Demo\DisplayDriver.o
_cursorX            0x2               Objects - Graphics Primitives Layer Demo\Primitive.o
_fontLastChar       0x2               Objects - Graphics Primitives Layer Demo\Primitive.o
_font               0x4               Objects - Graphics Primitives Layer Demo\Primitive.o
_lineType           0x2               Objects - Graphics Primitives Layer Demo\Primitive.o
_clipRight          0x2               Objects - Graphics Primitives Layer Demo\DisplayDriver.o
_clipBottom         0x2               Objects - Graphics Primitives Layer Demo\DisplayDriver.o
_page               0x1               Objects - Graphics Primitives Layer Demo\DisplayDriver.o
_clipTop            0x2               Objects - Graphics Primitives Layer Demo\DisplayDriver.o
_color              0x2               Objects - Graphics Primitives Layer Demo\DisplayDriver.o
_clipLeft           0x2               Objects - Graphics Primitives Layer Demo\DisplayDriver.o
_lineThickness      0x1               Objects - Graphics Primitives Layer Demo\Primitive.o

Memory Configuration

Name             Origin             Length             Attributes
kseg0_program_mem 0x9d000000         0x00080000         xr
kseg0_boot_mem   0x9fc00490         0x00000970
exception_mem    0x9fc01000         0x00001000
kseg1_boot_mem   0xbfc00000         0x00000490
debug_exec_mem   0xbfc02000         0x00000ff0
config3          0xbfc02ff0         0x00000004
config2          0xbfc02ff4         0x00000004
config1          0xbfc02ff8         0x00000004
config0          0xbfc02ffc         0x00000004
kseg1_data_mem   0xa0000000         0x00008000         w !x
sfrs             0xbf800000         0x00100000
*default*        0x00000000         0xffffffff

Linker script and memory map

LOAD C:/Program Files/Microchip/MPLAB C32/bin/../lib/gcc/pic32mx/3.4.4/../../../../pic32mx/lib/size/crt0.o
LOAD Objects - Graphics Primitives Layer Demo\MainDemo.o
LOAD Objects - Graphics Primitives Layer Demo\Pictures PIC32.o
LOAD Objects - Graphics Primitives Layer Demo\Font25PixelsHeight.o
LOAD Objects - Graphics Primitives Layer Demo\Window.o
LOAD Objects - Graphics Primitives Layer Demo\Button.o
LOAD Objects - Graphics Primitives Layer Demo\Chart.o
LOAD Objects - Graphics Primitives Layer Demo\CheckBox.o
LOAD Objects - Graphics Primitives Layer Demo\EditBox.o
LOAD Objects - Graphics Primitives Layer Demo\GOL.o
LOAD Objects - Graphics Primitives Layer Demo\GOLFontDefault.o
LOAD Objects - Graphics Primitives Layer Demo\Grid.o
LOAD Objects - Graphics Primitives Layer Demo\GroupBox.o
LOAD Objects - Graphics Primitives Layer Demo\ListBox.o
LOAD Objects - Graphics Primitives Layer Demo\Meter.o
LOAD Objects - Graphics Primitives Layer Demo\Picture.o
LOAD Objects - Graphics Primitives Layer Demo\Primitive.o
LOAD Objects - Graphics Primitives Layer Demo\ProgressBar.o
LOAD Objects - Graphics Primitives Layer Demo\RadioButton.o
LOAD Objects - Graphics Primitives Layer Demo\RoundDial.o
LOAD Objects - Graphics Primitives Layer Demo\Slider.o
LOAD Objects - Graphics Primitives Layer Demo\StaticText.o
LOAD Objects - Graphics Primitives Layer Demo\DisplayDriver.o
                0x00000001                __MPLAB_BUILD = 0x1
                0x00000fa0                _min_heap_size = 0xfa0
                0x00000800                _min_stack_size = 0x800
LOAD C:/Program Files/Microchip/MPLAB C32/bin/../lib/gcc/pic32mx/3.4.4/size\libgcc.a
START GROUP
LOAD C:/Program Files/Microchip/MPLAB C32/bin/../lib/gcc/pic32mx/3.4.4/../../../../pic32mx/lib/size\libc.a
LOAD C:/Program Files/Microchip/MPLAB C32/bin/../lib/gcc/pic32mx/3.4.4/../../../../pic32mx/lib/size\libm.a
LOAD C:/Program Files/Microchip/MPLAB C32/bin/../lib/gcc/pic32mx/3.4.4/../../../../pic32mx/lib/size\libe.a
LOAD C:/Program Files/Microchip/MPLAB C32/bin/../lib/gcc/pic32mx/3.4.4/../../../../pic32mx/lib/size\libmchp_peripheral.a
LOAD C:/Program Files/Microchip/MPLAB C32/bin/../lib/gcc/pic32mx/3.4.4/../../../../pic32mx/lib/size\libmchp_peripheral_32MX360F512L.a
END GROUP
LOAD C:/Program Files/Microchip/MPLAB C32/bin/../lib/gcc/pic32mx/3.4.4/size\libgcc.a
                0x00000400                PROVIDE (_min_stack_size, 0x400)
                0x00000000                PROVIDE (_min_heap_size, 0x0)
LOAD C:/Program Files/Microchip/MPLAB C32/bin/../lib/gcc/pic32mx/3.4.4/../../../../pic32mx/lib/./proc/32MX360F512L\processor.o
                0x00000001                PROVIDE (_vector_spacing, 0x1)
                0x9fc01000                _ebase_address = 0x9fc01000
                0xbfc00000                _RESET_ADDR = 0xbfc00000
                0xbfc00380                _BEV_EXCPT_ADDR = 0xbfc00380
                0xbfc00480                _DBG_EXCPT_ADDR = 0xbfc00480
                0xbfc02000                _DBG_CODE_ADDR = 0xbfc02000
                0x9fc01180                _GEN_EXCPT_ADDR = (_ebase_address + 0x180)

.config_BFC02FF0
 *(.config_BFC02FF0)

.config_BFC02FF4
                0xbfc02ff4        0x4
 *(.config_BFC02FF4)
 .config_BFC02FF4
                0xbfc02ff4        0x4 Objects - Graphics Primitives Layer Demo\MainDemo.o

.config_BFC02FF8
                0xbfc02ff8        0x4
 *(.config_BFC02FF8)
 .config_BFC02FF8
                0xbfc02ff8        0x4 Objects - Graphics Primitives Layer Demo\MainDemo.o

.config_BFC02FFC
                0xbfc02ffc        0x4
 *(.config_BFC02FFC)
 .config_BFC02FFC
                0xbfc02ffc        0x4 Objects - Graphics Primitives Layer Demo\MainDemo.o

.reset          0xbfc00000       0x10
 *(.reset)
 .reset         0xbfc00000       0x10 C:/Program Files/Microchip/MPLAB C32/bin/../lib/gcc/pic32mx/3.4.4/../../../../pic32mx/lib/size/crt0.o
                0xbfc00000                _reset

.bev_excpt      0xbfc00380       0x10
 *(.bev_handler)
 .bev_handler   0xbfc00380       0x10 C:/Program Files/Microchip/MPLAB C32/bin/../lib/gcc/pic32mx/3.4.4/../../../../pic32mx/lib/size/crt0.o

.dbg_excpt      0xbfc00480        0x0
                0xbfc00480                . = (. + DEFINED (_DEBUGGER)?0x8:0x0)

.dbg_code       0xbfc02000        0x0
                0xbfc02000                . = (. + DEFINED (_DEBUGGER)?0xff0:0x0)

.app_excpt      0x9fc01180       0x10
 *(.gen_handler)
 .gen_handler   0x9fc01180       0x10 C:/Program Files/Microchip/MPLAB C32/bin/../lib/gcc/pic32mx/3.4.4/../../../../pic32mx/lib/size/crt0.o

.vector_0       0x9fc01200        0x0
 *(.vector_0)
                0x00000001                ASSERT (((_vector_spacing == 0x0) || (SIZEOF (.vector_0) < (_vector_spacing << 0x5))), function at exception vector 0 too large)

.vector_1       0x9fc01220        0x0
 *(.vector_1)
                0x00000001                ASSERT (((_vector_spacing == 0x0) || (SIZEOF (.vector_1) < (_vector_spacing << 0x5))), function at exception vector 1 too large)

.vector_2       0x9fc01240        0x0
 *(.vector_2)
                0x00000001                ASSERT (((_vector_spacing == 0x0) || (SIZEOF (.vector_2) < (_vector_spacing << 0x5))), function at exception vector 2 too large)

.vector_3       0x9fc01260        0x0
 *(.vector_3)
                0x00000001                ASSERT (((_vector_spacing == 0x0) || (SIZEOF (.vector_3) < (_vector_spacing << 0x5))), function at exception vector 3 too large)

.vector_4       0x9fc01280        0x0
 *(.vector_4)
                0x00000001                ASSERT (((_vector_spacing == 0x0) || (SIZEOF (.vector_4) < (_vector_spacing << 0x5))), function at exception vector 4 too large)

.vector_5       0x9fc012a0        0x0
 *(.vector_5)
                0x00000001                ASSERT (((_vector_spacing == 0x0) || (SIZEOF (.vector_5) < (_vector_spacing << 0x5))), function at exception vector 5 too large)

.vector_6       0x9fc012c0        0x0
 *(.vector_6)
                0x00000001                ASSERT (((_vector_spacing == 0x0) || (SIZEOF (.vector_6) < (_vector_spacing << 0x5))), function at exception vector 6 too large)

.vector_7       0x9fc012e0        0x0
 *(.vector_7)
                0x00000001                ASSERT (((_vector_spacing == 0x0) || (SIZEOF (.vector_7) < (_vector_spacing << 0x5))), function at exception vector 7 too large)

.vector_8       0x9fc01300        0x0
 *(.vector_8)
                0x00000001                ASSERT (((_vector_spacing == 0x0) || (SIZEOF (.vector_8) < (_vector_spacing << 0x5))), function at exception vector 8 too large)

.vector_9       0x9fc01320        0x0
 *(.vector_9)
                0x00000001                ASSERT (((_vector_spacing == 0x0) || (SIZEOF (.vector_9) < (_vector_spacing << 0x5))), function at exception vector 9 too large)

.vector_10      0x9fc01340        0x0
 *(.vector_10)
                0x00000001                ASSERT (((_vector_spacing == 0x0) || (SIZEOF (.vector_10) < (_vector_spacing << 0x5))), function at exception vector 10 too large)

.vector_11      0x9fc01360        0x0
 *(.vector_11)
                0x00000001                ASSERT (((_vector_spacing == 0x0) || (SIZEOF (.vector_11) < (_vector_spacing << 0x5))), function at exception vector 11 too large)

.vector_12      0x9fc01380        0x0
 *(.vector_12)
                0x00000001                ASSERT (((_vector_spacing == 0x0) || (SIZEOF (.vector_12) < (_vector_spacing << 0x5))), function at exception vector 12 too large)

.vector_13      0x9fc013a0        0x0
 *(.vector_13)
                0x00000001                ASSERT (((_vector_spacing == 0x0) || (SIZEOF (.vector_13) < (_vector_spacing << 0x5))), function at exception vector 13 too large)

.vector_14      0x9fc013c0        0x0
 *(.vector_14)
                0x00000001                ASSERT (((_vector_spacing == 0x0) || (SIZEOF (.vector_14) < (_vector_spacing << 0x5))), function at exception vector 14 too large)

.vector_15      0x9fc013e0        0x0
 *(.vector_15)
                0x00000001                ASSERT (((_vector_spacing == 0x0) || (SIZEOF (.vector_15) < (_vector_spacing << 0x5))), function at exception vector 15 too large)

.vector_16      0x9fc01400        0x0
 *(.vector_16)
                0x00000001                ASSERT (((_vector_spacing == 0x0) || (SIZEOF (.vector_16) < (_vector_spacing << 0x5))), function at exception vector 16 too large)

.vector_17      0x9fc01420        0x0
 *(.vector_17)
                0x00000001                ASSERT (((_vector_spacing == 0x0) || (SIZEOF (.vector_17) < (_vector_spacing << 0x5))), function at exception vector 17 too large)

.vector_18      0x9fc01440        0x0
 *(.vector_18)
                0x00000001                ASSERT (((_vector_spacing == 0x0) || (SIZEOF (.vector_18) < (_vector_spacing << 0x5))), function at exception vector 18 too large)

.vector_19      0x9fc01460        0x0
 *(.vector_19)
                0x00000001                ASSERT (((_vector_spacing == 0x0) || (SIZEOF (.vector_19) < (_vector_spacing << 0x5))), function at exception vector 19 too large)

.vector_20      0x9fc01480        0x0
 *(.vector_20)
                0x00000001                ASSERT (((_vector_spacing == 0x0) || (SIZEOF (.vector_20) < (_vector_spacing << 0x5))), function at exception vector 20 too large)

.vector_21      0x9fc014a0        0x0
 *(.vector_21)
                0x00000001                ASSERT (((_vector_spacing == 0x0) || (SIZEOF (.vector_21) < (_vector_spacing << 0x5))), function at exception vector 21 too large)

.vector_22      0x9fc014c0        0x0
 *(.vector_22)
                0x00000001                ASSERT (((_vector_spacing == 0x0) || (SIZEOF (.vector_22) < (_vector_spacing << 0x5))), function at exception vector 22 too large)

.vector_23      0x9fc014e0        0x0
 *(.vector_23)
                0x00000001                ASSERT (((_vector_spacing == 0x0) || (SIZEOF (.vector_23) < (_vector_spacing << 0x5))), function at exception vector 23 too large)

.vector_24      0x9fc01500        0x0
 *(.vector_24)
                0x00000001                ASSERT (((_vector_spacing == 0x0) || (SIZEOF (.vector_24) < (_vector_spacing << 0x5))), function at exception vector 24 too large)

.vector_25      0x9fc01520        0x0
 *(.vector_25)
                0x00000001                ASSERT (((_vector_spacing == 0x0) || (SIZEOF (.vector_25) < (_vector_spacing << 0x5))), function at exception vector 25 too large)

.vector_26      0x9fc01540        0x0
 *(.vector_26)
                0x00000001                ASSERT (((_vector_spacing == 0x0) || (SIZEOF (.vector_26) < (_vector_spacing << 0x5))), function at exception vector 26 too large)

.vector_27      0x9fc01560        0x0
 *(.vector_27)
                0x00000001                ASSERT (((_vector_spacing == 0x0) || (SIZEOF (.vector_27) < (_vector_spacing << 0x5))), function at exception vector 27 too large)

.vector_28      0x9fc01580        0x0
 *(.vector_28)
                0x00000001                ASSERT (((_vector_spacing == 0x0) || (SIZEOF (.vector_28) < (_vector_spacing << 0x5))), function at exception vector 28 too large)

.vector_29      0x9fc015a0        0x0
 *(.vector_29)
                0x00000001                ASSERT (((_vector_spacing == 0x0) || (SIZEOF (.vector_29) < (_vector_spacing << 0x5))), function at exception vector 29 too large)

.vector_30      0x9fc015c0        0x0
 *(.vector_30)
                0x00000001                ASSERT (((_vector_spacing == 0x0) || (SIZEOF (.vector_30) < (_vector_spacing << 0x5))), function at exception vector 30 too large)

.vector_31      0x9fc015e0        0x0
 *(.vector_31)
                0x00000001                ASSERT (((_vector_spacing == 0x0) || (SIZEOF (.vector_31) < (_vector_spacing << 0x5))), function at exception vector 31 too large)

.vector_32      0x9fc01600        0x0
 *(.vector_32)
                0x00000001                ASSERT (((_vector_spacing == 0x0) || (SIZEOF (.vector_32) < (_vector_spacing << 0x5))), function at exception vector 32 too large)

.vector_33      0x9fc01620        0x0
 *(.vector_33)
                0x00000001                ASSERT (((_vector_spacing == 0x0) || (SIZEOF (.vector_33) < (_vector_spacing << 0x5))), function at exception vector 33 too large)

.vector_34      0x9fc01640        0x0
 *(.vector_34)
                0x00000001                ASSERT (((_vector_spacing == 0x0) || (SIZEOF (.vector_34) < (_vector_spacing << 0x5))), function at exception vector 34 too large)

.vector_35      0x9fc01660        0x0
 *(.vector_35)
                0x00000001                ASSERT (((_vector_spacing == 0x0) || (SIZEOF (.vector_35) < (_vector_spacing << 0x5))), function at exception vector 35 too large)

.vector_36      0x9fc01680        0x0
 *(.vector_36)
                0x00000001                ASSERT (((_vector_spacing == 0x0) || (SIZEOF (.vector_36) < (_vector_spacing << 0x5))), function at exception vector 36 too large)

.vector_37      0x9fc016a0        0x0
 *(.vector_37)
                0x00000001                ASSERT (((_vector_spacing == 0x0) || (SIZEOF (.vector_37) < (_vector_spacing << 0x5))), function at exception vector 37 too large)

.vector_38      0x9fc016c0        0x0
 *(.vector_38)
                0x00000001                ASSERT (((_vector_spacing == 0x0) || (SIZEOF (.vector_38) < (_vector_spacing << 0x5))), function at exception vector 38 too large)

.vector_39      0x9fc016e0        0x0
 *(.vector_39)
                0x00000001                ASSERT (((_vector_spacing == 0x0) || (SIZEOF (.vector_39) < (_vector_spacing << 0x5))), function at exception vector 39 too large)

.vector_40      0x9fc01700        0x0
 *(.vector_40)
                0x00000001                ASSERT (((_vector_spacing == 0x0) || (SIZEOF (.vector_40) < (_vector_spacing << 0x5))), function at exception vector 40 too large)

.vector_41      0x9fc01720        0x0
 *(.vector_41)
                0x00000001                ASSERT (((_vector_spacing == 0x0) || (SIZEOF (.vector_41) < (_vector_spacing << 0x5))), function at exception vector 41 too large)

.vector_42      0x9fc01740        0x0
 *(.vector_42)
                0x00000001                ASSERT (((_vector_spacing == 0x0) || (SIZEOF (.vector_42) < (_vector_spacing << 0x5))), function at exception vector 42 too large)

.vector_43      0x9fc01760        0x0
 *(.vector_43)
                0x00000001                ASSERT (((_vector_spacing == 0x0) || (SIZEOF (.vector_43) < (_vector_spacing << 0x5))), function at exception vector 43 too large)

.vector_44      0x9fc01780        0x0
 *(.vector_44)
                0x00000001                ASSERT (((_vector_spacing == 0x0) || (SIZEOF (.vector_44) < (_vector_spacing << 0x5))), function at exception vector 44 too large)

.vector_45      0x9fc017a0        0x0
 *(.vector_45)
                0x00000001                ASSERT (((_vector_spacing == 0x0) || (SIZEOF (.vector_45) < (_vector_spacing << 0x5))), function at exception vector 45 too large)

.vector_46      0x9fc017c0        0x0
 *(.vector_46)
                0x00000001                ASSERT (((_vector_spacing == 0x0) || (SIZEOF (.vector_46) < (_vector_spacing << 0x5))), function at exception vector 46 too large)

.vector_47      0x9fc017e0        0x0
 *(.vector_47)
                0x00000001                ASSERT (((_vector_spacing == 0x0) || (SIZEOF (.vector_47) < (_vector_spacing << 0x5))), function at exception vector 47 too large)

.vector_48      0x9fc01800        0x0
 *(.vector_48)
                0x00000001                ASSERT (((_vector_spacing == 0x0) || (SIZEOF (.vector_48) < (_vector_spacing << 0x5))), function at exception vector 48 too large)

.vector_49      0x9fc01820        0x0
 *(.vector_49)
                0x00000001                ASSERT (((_vector_spacing == 0x0) || (SIZEOF (.vector_49) < (_vector_spacing << 0x5))), function at exception vector 49 too large)

.vector_50      0x9fc01840        0x0
 *(.vector_50)
                0x00000001                ASSERT (((_vector_spacing == 0x0) || (SIZEOF (.vector_50) < (_vector_spacing << 0x5))), function at exception vector 50 too large)

.vector_51      0x9fc01860        0x0
 *(.vector_51)
                0x00000001                ASSERT (((_vector_spacing == 0x0) || (SIZEOF (.vector_51) < (_vector_spacing << 0x5))), function at exception vector 51 too large)

.vector_52      0x9fc01880        0x0
 *(.vector_52)
                0x00000001                ASSERT (((_vector_spacing == 0x0) || (SIZEOF (.vector_52) < (_vector_spacing << 0x5))), function at exception vector 52 too large)

.vector_53      0x9fc018a0        0x0
 *(.vector_53)
                0x00000001                ASSERT (((_vector_spacing == 0x0) || (SIZEOF (.vector_53) < (_vector_spacing << 0x5))), function at exception vector 53 too large)

.vector_54      0x9fc018c0        0x0
 *(.vector_54)
                0x00000001                ASSERT (((_vector_spacing == 0x0) || (SIZEOF (.vector_54) < (_vector_spacing << 0x5))), function at exception vector 54 too large)

.vector_55      0x9fc018e0        0x0
 *(.vector_55)
                0x00000001                ASSERT (((_vector_spacing == 0x0) || (SIZEOF (.vector_55) < (_vector_spacing << 0x5))), function at exception vector 55 too large)

.vector_56      0x9fc01900        0x0
 *(.vector_56)
                0x00000001                ASSERT (((_vector_spacing == 0x0) || (SIZEOF (.vector_56) < (_vector_spacing << 0x5))), function at exception vector 56 too large)

.vector_57      0x9fc01920        0x0
 *(.vector_57)
                0x00000001                ASSERT (((_vector_spacing == 0x0) || (SIZEOF (.vector_57) < (_vector_spacing << 0x5))), function at exception vector 57 too large)

.vector_58      0x9fc01940        0x0
 *(.vector_58)
                0x00000001                ASSERT (((_vector_spacing == 0x0) || (SIZEOF (.vector_58) < (_vector_spacing << 0x5))), function at exception vector 58 too large)

.vector_59      0x9fc01960        0x0
 *(.vector_59)
                0x00000001                ASSERT (((_vector_spacing == 0x0) || (SIZEOF (.vector_59) < (_vector_spacing << 0x5))), function at exception vector 59 too large)

.vector_60      0x9fc01980        0x0
 *(.vector_60)
                0x00000001                ASSERT (((_vector_spacing == 0x0) || (SIZEOF (.vector_60) < (_vector_spacing << 0x5))), function at exception vector 60 too large)

.vector_61      0x9fc019a0        0x0
 *(.vector_61)
                0x00000001                ASSERT (((_vector_spacing == 0x0) || (SIZEOF (.vector_61) < (_vector_spacing << 0x5))), function at exception vector 61 too large)

.vector_62      0x9fc019c0        0x0
 *(.vector_62)
                0x00000001                ASSERT (((_vector_spacing == 0x0) || (SIZEOF (.vector_62) < (_vector_spacing << 0x5))), function at exception vector 62 too large)

.vector_63      0x9fc019e0        0x0
 *(.vector_63)
                0x00000001                ASSERT (((_vector_spacing == 0x0) || (SIZEOF (.vector_63) < (_vector_spacing << 0x5))), function at exception vector 63 too large)

.startup        0x9fc00490      0x1e0
 *(.startup)
 .startup       0x9fc00490      0x1e0 C:/Program Files/Microchip/MPLAB C32/bin/../lib/gcc/pic32mx/3.4.4/../../../../pic32mx/lib/size/crt0.o

.text           0x9d000000    0x7429c
                0x9d000000                _text_begin = .
 *(.text .stub .text.* .gnu.linkonce.t.*)
 .text          0x9d000000       0x18 C:/Program Files/Microchip/MPLAB C32/bin/../lib/gcc/pic32mx/3.4.4/../../../../pic32mx/lib/size/crt0.o
 .text          0x9d000018      0x840 Objects - Graphics Primitives Layer Demo\MainDemo.o
                0x9d000018                main
 .text          0x9d000858     0x14a4 Objects - Graphics Primitives Layer Demo\Primitive.o
                0x9d001224                Bevel
                0x9d0018e8                DrawPoly
                0x9d001bbc                OutTextXY
                0x9d00168c                FillBevel
                0x9d001b58                OutText
                0x9d001970                SetFont
                0x9d001cdc                GetImageHeight
                0x9d001cbc                GetImageWidth
                0x9d000ee0                Line
                0x9d000898                Arc
                0x9d001c9c                GetTextHeight
                0x9d001c10                GetTextWidth
                0x9d000858                InitGraph
                0x9d0019a0                OutChar
 .text          0x9d001cfc     0x1e58 Objects - Graphics Primitives Layer Demo\DisplayDriver.o
                0x9d0038b8                ssd1928_FloatWndInit
                0x9d001cfc                DelayMs
                0x9d003088                PutImage16BPP
                0x9d00229c                GetRegW
                0x9d003264                PutImage
                0x9d003a00                ssd1928_MainWndInit
                0x9d001eb0                SetRegB
                0x9d003b14                ssd1928_MainWndEnable
                0x9d002594                GetPixel
                0x9d001d84                SetAddress
                0x9d002048                GetReg
                0x9d0022dc                SetRegW
                0x9d0039c0                ssd1928_FloatWndEnable
                0x9d0023c8                GPIO_SPCLK
                0x9d0023f0                GPIO_SPDAT
                0x9d003ab0                ssd1928_FocusWnd
                0x9d002320                SetRegL
                0x9d002914                ClearDevice
                0x9d0023a0                GPIO_SPENA
                0x9d002a24                PutImage1BPP
                0x9d00331c                SPI_Write
                0x9d002418                GPIO_SPRESET
                0x9d003400                ResetDevice
                0x9d002760                Bar
                0x9d002440                PutPixel
                0x9d003388                SPI_SetReg
                0x9d002c3c                PutImage4BPP
                0x9d002364                GetRegL
                0x9d002e6c                PutImage8BPP
 .text          0x9d003b54      0x168 C:/Program Files/Microchip/MPLAB C32/bin/../lib/gcc/pic32mx/3.4.4/../../../../pic32mx/lib/size\libc.a(memcpy.o)
                0x9d003b54                memcpy
 .text.general_exception
                0x9d003cbc       0xd0 C:/Program Files/Microchip/MPLAB C32/bin/../lib/gcc/pic32mx/3.4.4/../../../../pic32mx/lib/size\libc.a(general-exception.o)
                0x9d003cbc                _general_exception_context
 .text.exit     0x9d003d8c       0x9c C:/Program Files/Microchip/MPLAB C32/bin/../lib/gcc/pic32mx/3.4.4/../../../../pic32mx/lib/size\libc.a(exit.o)
                0x9d003d8c                exit
 .text._filbuf_simple
                0x9d003e28       0x48 C:/Program Files/Microchip/MPLAB C32/bin/../lib/gcc/pic32mx/3.4.4/../../../../pic32mx/lib/size\libc.a(_iobfuncs.o)
                0x9d003e28                _filbuf_simple
 .text._fflush_simple
                0x9d003e70       0x6c C:/Program Files/Microchip/MPLAB C32/bin/../lib/gcc/pic32mx/3.4.4/../../../../pic32mx/lib/size\libc.a(_iobfuncs.o)
                0x9d003e70                _fflush_simple
 .text._flsbuf_simple
                0x9d003edc       0xdc C:/Program Files/Microchip/MPLAB C32/bin/../lib/gcc/pic32mx/3.4.4/../../../../pic32mx/lib/size\libc.a(_iobfuncs.o)
                0x9d003edc                _flsbuf_simple
 .text._fwrite_simple
                0x9d003fb8       0x84 C:/Program Files/Microchip/MPLAB C32/bin/../lib/gcc/pic32mx/3.4.4/../../../../pic32mx/lib/size\libc.a(_iobfuncs.o)
                0x9d003fb8                _fwrite_simple
 .text._fsync_simple
                0x9d00403c       0x34 C:/Program Files/Microchip/MPLAB C32/bin/../lib/gcc/pic32mx/3.4.4/../../../../pic32mx/lib/size\libc.a(_iobfuncs.o)
                0x9d00403c                _fsync_simple
 .text._weak_pthread_mutex_init
                0x9d004070        0x8 C:/Program Files/Microchip/MPLAB C32/bin/../lib/gcc/pic32mx/3.4.4/../../../../pic32mx/lib/size\libc.a(stubs.o)
                0x9d004070                _weak_pthread_mutex_init
                0x9d004070                pthread_mutex_init
 .text._weak_pthread_mutex_destroy
                0x9d004078        0x8 C:/Program Files/Microchip/MPLAB C32/bin/../lib/gcc/pic32mx/3.4.4/../../../../pic32mx/lib/size\libc.a(stubs.o)
                0x9d004078                _weak_pthread_mutex_destroy
                0x9d004078                pthread_mutex_destroy
 .text._weak_pthread_mutex_lock
                0x9d004080        0x8 C:/Program Files/Microchip/MPLAB C32/bin/../lib/gcc/pic32mx/3.4.4/../../../../pic32mx/lib/size\libc.a(stubs.o)
                0x9d004080                _weak_pthread_mutex_lock
                0x9d004080                pthread_mutex_lock
 .text._weak_pthread_mutex_trylock
                0x9d004088        0x8 C:/Program Files/Microchip/MPLAB C32/bin/../lib/gcc/pic32mx/3.4.4/../../../../pic32mx/lib/size\libc.a(stubs.o)
                0x9d004088                _weak_pthread_mutex_trylock
                0x9d004088                pthread_mutex_trylock
 .text._weak_pthread_mutex_unlock
                0x9d004090        0x8 C:/Program Files/Microchip/MPLAB C32/bin/../lib/gcc/pic32mx/3.4.4/../../../../pic32mx/lib/size\libc.a(stubs.o)
                0x9d004090                _weak_pthread_mutex_unlock
                0x9d004090                pthread_mutex_unlock
 .text._weak_pthread_mutex_setname_np
                0x9d004098        0x8 C:/Program Files/Microchip/MPLAB C32/bin/../lib/gcc/pic32mx/3.4.4/../../../../pic32mx/lib/size\libc.a(stubs.o)
                0x9d004098                pthread_mutex_setname_np
                0x9d004098                _weak_pthread_mutex_setname_np
 .text._weak_pthread_mutexattr_init
                0x9d0040a0        0x8 C:/Program Files/Microchip/MPLAB C32/bin/../lib/gcc/pic32mx/3.4.4/../../../../pic32mx/lib/size\libc.a(stubs.o)
                0x9d0040a0                _weak_pthread_mutexattr_init
                0x9d0040a0                pthread_mutexattr_init
 .text._weak_pthread_mutexattr_destroy
                0x9d0040a8        0x8 C:/Program Files/Microchip/MPLAB C32/bin/../lib/gcc/pic32mx/3.4.4/../../../../pic32mx/lib/size\libc.a(stubs.o)
                0x9d0040a8                pthread_mutexattr_destroy
                0x9d0040a8                _weak_pthread_mutexattr_destroy
 .text._weak_pthread_mutexattr_setname_np
                0x9d0040b0        0x8 C:/Program Files/Microchip/MPLAB C32/bin/../lib/gcc/pic32mx/3.4.4/../../../../pic32mx/lib/size\libc.a(stubs.o)
                0x9d0040b0                _weak_pthread_mutexattr_setname_np
                0x9d0040b0                pthread_mutexattr_setname_np
 .text._weak_pthread_mutexattr_settype_np
                0x9d0040b8        0x8 C:/Program Files/Microchip/MPLAB C32/bin/../lib/gcc/pic32mx/3.4.4/../../../../pic32mx/lib/size\libc.a(stubs.o)
                0x9d0040b8                _weak_pthread_mutexattr_settype_np
                0x9d0040b8                pthread_mutexattr_settype_np
 .text._weak_pthread_sysconf_np
                0x9d0040c0        0x8 C:/Program Files/Microchip/MPLAB C32/bin/../lib/gcc/pic32mx/3.4.4/../../../../pic32mx/lib/size\libc.a(stubs.o)
                0x9d0040c0                _weak_pthread_sysconf_np
                0x9d0040c0                pthread_sysconf_np
 .text._weak_pthread_sigdisable_np
                0x9d0040c8        0x8 C:/Program Files/Microchip/MPLAB C32/bin/../lib/gcc/pic32mx/3.4.4/../../../../pic32mx/lib/size\libc.a(stubs.o)
                0x9d0040c8                _weak_pthread_sigdisable_np
                0x9d0040c8                pthread_sigdisable_np
 .text._weak_pthread_sigrestore_np
                0x9d0040d0        0x8 C:/Program Files/Microchip/MPLAB C32/bin/../lib/gcc/pic32mx/3.4.4/../../../../pic32mx/lib/size\libc.a(stubs.o)
                0x9d0040d0                pthread_sigrestore_np
                0x9d0040d0                _weak_pthread_sigrestore_np
 .text._weak__pthread_cleanup_push
                0x9d0040d8        0x8 C:/Program Files/Microchip/MPLAB C32/bin/../lib/gcc/pic32mx/3.4.4/../../../../pic32mx/lib/size\libc.a(stubs.o)
                0x9d0040d8                _weak__pthread_cleanup_push
                0x9d0040d8                _pthread_cleanup_push
 .text._weak__pthread_cleanup_pop
                0x9d0040e0        0x8 C:/Program Files/Microchip/MPLAB C32/bin/../lib/gcc/pic32mx/3.4.4/../../../../pic32mx/lib/size\libc.a(stubs.o)
                0x9d0040e0                _pthread_cleanup_pop
                0x9d0040e0                _weak__pthread_cleanup_pop
 .text._weak__pthread_cleanup_push_defer
                0x9d0040e8        0x8 C:/Program Files/Microchip/MPLAB C32/bin/../lib/gcc/pic32mx/3.4.4/../../../../pic32mx/lib/size\libc.a(stubs.o)
                0x9d0040e8                _weak__pthread_cleanup_push_defer
                0x9d0040e8                _pthread_cleanup_push_defer
 .text._weak__pthread_cleanup_pop_restore
                0x9d0040f0        0x8 C:/Program Files/Microchip/MPLAB C32/bin/../lib/gcc/pic32mx/3.4.4/../../../../pic32mx/lib/size\libc.a(stubs.o)
                0x9d0040f0                _pthread_cleanup_pop_restore
                0x9d0040f0                _weak__pthread_cleanup_pop_restore
 .text._weak_pthread_once
                0x9d0040f8       0x2c C:/Program Files/Microchip/MPLAB C32/bin/../lib/gcc/pic32mx/3.4.4/../../../../pic32mx/lib/size\libc.a(stubs.o)
                0x9d0040f8                _weak_pthread_once
                0x9d0040f8                pthread_once
                0x9d0040f8                _pthread_once
 .text._weak_pthread_key_create
                0x9d004124        0x8 C:/Program Files/Microchip/MPLAB C32/bin/../lib/gcc/pic32mx/3.4.4/../../../../pic32mx/lib/size\libc.a(stubs.o)
                0x9d004124                pthread_key_create
                0x9d004124                _weak_pthread_key_create
 .text._weak_pthread_setspecific
                0x9d00412c        0x8 C:/Program Files/Microchip/MPLAB C32/bin/../lib/gcc/pic32mx/3.4.4/../../../../pic32mx/lib/size\libc.a(stubs.o)
                0x9d00412c                _weak_pthread_setspecific
                0x9d00412c                pthread_setspecific
 .text._weak_pthread_getspecific
                0x9d004134        0x8 C:/Program Files/Microchip/MPLAB C32/bin/../lib/gcc/pic32mx/3.4.4/../../../../pic32mx/lib/size\libc.a(stubs.o)
                0x9d004134                pthread_getspecific
                0x9d004134                _weak_pthread_getspecific
 .text._weak__libc_private_storage
                0x9d00413c        0x8 C:/Program Files/Microchip/MPLAB C32/bin/../lib/gcc/pic32mx/3.4.4/../../../../pic32mx/lib/size\libc.a(stubs.o)
                0x9d00413c                _libc_private_storage
                0x9d00413c                _weak__libc_private_storage
 .text._general_exception_handler
                0x9d004144        0x8 C:/Program Files/Microchip/MPLAB C32/bin/../lib/gcc/pic32mx/3.4.4/../../../../pic32mx/lib/size\libc.a(default-general-exception-handler.o)
                0x9d004144                _general_exception_handler
 .text._bootstrap_exception_handler
                0x9d00414c        0x8 C:/Program Files/Microchip/MPLAB C32/bin/../lib/gcc/pic32mx/3.4.4/../../../../pic32mx/lib/size\libc.a(default-bootstrap-exception-handler.o)
                0x9d00414c                _bootstrap_exception_handler
 .text._on_reset
                0x9d004154        0x8 C:/Program Files/Microchip/MPLAB C32/bin/../lib/gcc/pic32mx/3.4.4/../../../../pic32mx/lib/size\libc.a(default-on-reset.o)
                0x9d004154                _on_reset
 .text._on_bootstrap
                0x9d00415c        0x8 C:/Program Files/Microchip/MPLAB C32/bin/../lib/gcc/pic32mx/3.4.4/../../../../pic32mx/lib/size\libc.a(default-on-bootstrap.o)
                0x9d00415c                _on_bootstrap
 .text          0x9d004164       0x18 C:/Program Files/Microchip/MPLAB C32/bin/../lib/gcc/pic32mx/3.4.4/../../../../pic32mx/lib/size\libc.a(default-nmi-handler.o)
                0x9d004164                _nmi_handler
 .text._mon_getc
                0x9d00417c        0x8 C:/Program Files/Microchip/MPLAB C32/bin/../lib/gcc/pic32mx/3.4.4/../../../../pic32mx/lib/size\libc.a(_mon_getc.o)
                0x9d00417c                _mon_getc
 .text._mon_write
                0x9d004184       0x4c C:/Program Files/Microchip/MPLAB C32/bin/../lib/gcc/pic32mx/3.4.4/../../../../pic32mx/lib/size\libc.a(_mon_write.o)
                0x9d004184                _mon_write
 .text._exit    0x9d0041d0        0x8 C:/Program Files/Microchip/MPLAB C32/bin/../lib/gcc/pic32mx/3.4.4/../../../../pic32mx/lib/size\libc.a(_exit.o)
                0x9d0041d0                _exit
 .text._mon_putc
                0x9d0041d8       0x28 C:/Program Files/Microchip/MPLAB C32/bin/../lib/gcc/pic32mx/3.4.4/../../../../pic32mx/lib/size\libc.a(_mon_putc.o)
                0x9d0041d8                _mon_putc
 .text.INTDisableInterrupts
                0x9d004200        0x8 C:/Program Files/Microchip/MPLAB C32/bin/../lib/gcc/pic32mx/3.4.4/../../../../pic32mx/lib/size\libmchp_peripheral.a(int_disable_interrupts_lib.o)
                0x9d004200                INTDisableInterrupts
 .text.INTEnableSystemMultiVectoredInt
                0x9d004208       0x34 C:/Program Files/Microchip/MPLAB C32/bin/../lib/gcc/pic32mx/3.4.4/../../../../pic32mx/lib/size\libmchp_peripheral.a(int_enable_mv_int_lib.o)
                0x9d004208                INTEnableSystemMultiVectoredInt
 .text.INTRestoreInterrupts
                0x9d00423c       0x1c C:/Program Files/Microchip/MPLAB C32/bin/../lib/gcc/pic32mx/3.4.4/../../../../pic32mx/lib/size\libmchp_peripheral.a(int_restore_interrupts_lib.o)
                0x9d00423c                INTRestoreInterrupts
 .text.OpenCoreTimer
                0x9d004258        0xc C:/Program Files/Microchip/MPLAB C32/bin/../lib/gcc/pic32mx/3.4.4/../../../../pic32mx/lib/size\libmchp_peripheral.a(open_core_timer_lib.o)
                0x9d004258                OpenCoreTimer
 .text.CheKseg0CacheOff
                0x9d004264       0x18 C:/Program Files/Microchip/MPLAB C32/bin/../lib/gcc/pic32mx/3.4.4/../../../../pic32mx/lib/size\libmchp_peripheral.a(pcache.o)
                0x9d004264                CheKseg0CacheOff
 .text.CheKseg0CacheOn
                0x9d00427c       0x18 C:/Program Files/Microchip/MPLAB C32/bin/../lib/gcc/pic32mx/3.4.4/../../../../pic32mx/lib/size\libmchp_peripheral.a(pcache.o)
                0x9d00427c                CheKseg0CacheOn
 .text.INTEnableInterrupts
                0x9d004294        0x8 C:/Program Files/Microchip/MPLAB C32/bin/../lib/gcc/pic32mx/3.4.4/../../../../pic32mx/lib/size\libmchp_peripheral.a(int_enable_interrupts_lib.o)
                0x9d004294                INTEnableInterrupts
 .text          0x9d00429c    0x70000 C:/Program Files/Microchip/MPLAB C32/bin/../lib/gcc/pic32mx/3.4.4/../../../../pic32mx/lib/./proc/32MX360F512L\processor.o
 *(.text.*personality*)
 *(.gnu.warning)
 *(.mips16.fn.*)
 *(.mips16.call.*)
                0x9d07429c                _text_end = .
                *undef*                   ASSERT ((SIZEOF (.C32_EDITION_LIMITED_TO_64KB_EVALUATION) < (0x80000 - (((((((((SIZEOF (.text) + SIZEOF (.rodata)) + SIZEOF (.sdata2)) + SIZEOF (.sbss2)) + SIZEOF (.data)) + SIZEOF (.got)) + SIZEOF (.sdata)) + SIZEOF (.lit8)) + SIZEOF (.lit4)) + SIZEOF (.ramfunc)))), HINT: This application may be too large for this 64KB-limited edition of the MPLAB C32 Compiler. Visit http://www.microchip.com/c32 to upgrade to full version.)
                *undef*                   ASSERT ((SIZEOF (.C32_EDITION_LIMITED_TO_16KB_EVALUATION) < (0x80000 - (((((((((SIZEOF (.text) + SIZEOF (.rodata)) + SIZEOF (.sdata2)) + SIZEOF (.sbss2)) + SIZEOF (.data)) + SIZEOF (.got)) + SIZEOF (.sdata)) + SIZEOF (.lit8)) + SIZEOF (.lit4)) + SIZEOF (.ramfunc)))), HINT: This application may be too large for this 16KB-limited edition of the MPLAB C32 Compiler. Visit http://www.microchip.com/c32 to upgrade to full version.)
                *undef*                   ASSERT ((SIZEOF (.C32_EDITION_SIZELIMITED_EVALUATION) < (0x80000 - (((((((((SIZEOF (.text) + SIZEOF (.rodata)) + SIZEOF (.sdata2)) + SIZEOF (.sbss2)) + SIZEOF (.data)) + SIZEOF (.got)) + SIZEOF (.sdata)) + SIZEOF (.lit8)) + SIZEOF (.lit4)) + SIZEOF (.ramfunc)))), HINT: This application may be too large for this size-limited edition of the MPLAB C32 Compiler. Visit http://www.microchip.com/c32 to upgrade to full version.)

.rodata         0x9d07429c     0x9db0
 *(.rodata .rodata.* .gnu.linkonce.r.*)
 .rodata        0x9d07429c       0x14 Objects - Graphics Primitives Layer Demo\MainDemo.o
 .rodata.str1.4
                0x9d0742b0       0x2c Objects - Graphics Primitives Layer Demo\MainDemo.o
 .rodata        0x9d0742dc     0x8ac8 Objects - Graphics Primitives Layer Demo\Pictures PIC32.o
                0x9d07828c                L17867
                0x9d078284                flower8bit
                0x9d075af0                flower4bit
                0x9d07cd9c                flower16bit
                0x9d0742dc                L20864
                0x9d075af8                L18630
                0x9d0747cc                L27635
                0x9d0747c4                flower1bit
 .rodata        0x9d07cda4     0x122c Objects - Graphics Primitives Layer Demo\Font25PixelsHeight.o
                0x9d07cda4                L25
                0x9d07dfc8                Font25
 .rodata        0x9d07dfd0       0x68 Objects - Graphics Primitives Layer Demo\Primitive.o
 .rodata        0x9d07e038       0x14 C:/Program Files/Microchip/MPLAB C32/bin/../lib/gcc/pic32mx/3.4.4/../../../../pic32mx/lib/size\libc.a(_iobdata.o)
                0x9d07e038                _io_funcs
 *(.rodata1)
                0x9d07e04c                . = ALIGN (0x4)

.sdata2         0x9d07e04c        0x0
 *(.sdata2 .sdata2.* .gnu.linkonce.s2.*)
                0x9d07e04c                . = ALIGN (0x4)

.sbss2          0x9d07e04c        0x0
 *(.sbss2 .sbss2.* .gnu.linkonce.sb2.*)
                0x9d07e04c                . = ALIGN (0x4)

.eh_frame_hdr
 *(.eh_frame_hdr)

.eh_frame
 *(.eh_frame)

.dbg_data       0xa0000000        0x0
                0xa0000000                . = (. + DEFINED (_DEBUGGER)?0x200:0x0)

.data           0xa0000000       0xf4 load address 0x9d07e04c
                0xa0000000                _data_begin = .
 *(.data .data.* .gnu.linkonce.d.*)
 .data          0xa0000000       0x20 C:/Program Files/Microchip/MPLAB C32/bin/../lib/gcc/pic32mx/3.4.4/../../../../pic32mx/lib/size\libc.a(exit.o)
                0xa0000000                __exfun_mx
 .data          0xa0000020       0xd4 C:/Program Files/Microchip/MPLAB C32/bin/../lib/gcc/pic32mx/3.4.4/../../../../pic32mx/lib/size\libc.a(_iobdata.o)
 *(.gnu.linkonce.d.*personality*)
 *(.data1)
                0x9d07e04c                _data_image_begin = LOADADDR (.data)

.eh_frame
 *(.eh_frame)
                0xa00080f0                _gp = (ALIGN (0x10) + 0x7ff0)

.got            0xa00000f4        0x0 load address 0x9d07e140
 *(.got.plt)
 *(.got)

.sdata          0xa00000f4        0x8 load address 0x9d07e140
                0xa00000f4                _sdata_begin = .
 *(.sdata .sdata.* .gnu.linkonce.s.*)
 .sdata         0xa00000f4        0x1 Objects - Graphics Primitives Layer Demo\Primitive.o
 *fill*         0xa00000f5        0x3 00
 .sdata         0xa00000f8        0x4 C:/Program Files/Microchip/MPLAB C32/bin/../lib/gcc/pic32mx/3.4.4/../../../../pic32mx/lib/size\libc.a(_iobdata.o)
                0xa00000f8                _libc_data
                0xa00000fc                _sdata_end = .

.lit8           0xa00000fc        0x0 load address 0x9d07e148
 *(.lit8)

.lit4           0xa00000fc        0x0 load address 0x9d07e148
 *(.lit4)
                0xa00000fc                . = ALIGN (0x4)
                0xa00000fc                _data_end = .
                0xa00000fc                _bss_begin = .

.sbss           0xa00000fc       0x64
                0xa00000fc                _sbss_begin = .
 *(.dynsbss)
 *(.sbss .sbss.* .gnu.linkonce.sb.*)
 .sbss          0xa00000fc       0x34 Objects - Graphics Primitives Layer Demo\Primitive.o
 .sbss          0xa0000130        0x1 Objects - Graphics Primitives Layer Demo\DisplayDriver.o
                0xa0000130                _gpioStatus
 *fill*         0xa0000131        0x3 00
 .sbss          0xa0000134        0x4 C:/Program Files/Microchip/MPLAB C32/bin/../lib/gcc/pic32mx/3.4.4/../../../../pic32mx/lib/size\libc.a(errno.o)
                0xa0000134                errno
 *(.scommon)
 .scommon       0xa0000138       0x13 Objects - Graphics Primitives Layer Demo\Primitive.o
                0xa0000138                _cursorY
                0xa000013a                _fontOrientation
                0xa000013c                _fontFirstChar
                0xa000013e                _fontHeight
                0xa0000140                _cursorX
                0xa0000142                _fontLastChar
                0xa0000144                _font
                0xa0000148                _lineType
                0xa000014a                _lineThickness
 *fill*         0xa000014b        0x1 00
 .scommon       0xa000014c       0x14 Objects - Graphics Primitives Layer Demo\DisplayDriver.o
                0xa000014c                _clipRgn
                0xa0000150                _line_mem_pitch
                0xa0000154                _clipRight
                0xa0000156                _clipBottom
                0xa0000158                _page
                0xa000015a                _clipTop
                0xa000015c                _color
                0xa000015e                _clipLeft
                0xa0000160                _sbss_end = .

.bss            0xa0000160      0x10c
 *(.dynbss)
 *(.bss .bss.* .gnu.linkonce.b.*)
 .bss           0xa0000160       0x88 C:/Program Files/Microchip/MPLAB C32/bin/../lib/gcc/pic32mx/3.4.4/../../../../pic32mx/lib/size\libc.a(_iobdata.o)
 .bss           0xa00001e8       0x80 C:/Program Files/Microchip/MPLAB C32/bin/../lib/gcc/pic32mx/3.4.4/../../../../pic32mx/lib/size\libc.a(_iobfuncs.o)
 .bss           0xa0000268        0x4 C:/Program Files/Microchip/MPLAB C32/bin/../lib/gcc/pic32mx/3.4.4/../../../../pic32mx/lib/size\libc.a(stubs.o)
                0xa0000268                __isthreaded
 *(COMMON)
                0xa000026c                . = ALIGN (0x4)
                0xa000026c                . = ALIGN (0x4)
                0xa000026c                _end = .
                0xa000026c                _bss_end = .

.heap           0xa000026c      0xfa0
                0xa000026c                _heap = .
                0xa000120c                . = (. + _min_heap_size)
 *fill*         0xa000026c      0xfa0 00

.stack          0xa000120c      0x800
                0xa0001a0c                . = (. + _min_stack_size)
 *fill*         0xa000120c      0x800 00

.ramfunc        0xa0002000        0x0 load address 0x9d07e148
                0xa0002000                _ramfunc_begin = .
 *(.ramfunc .ramfunc.*)
                0xa0002000                . = ALIGN (0x4)
                0xa0002000                _ramfunc_end = .
                0x9d07e148                _ramfunc_image_begin = LOADADDR (.ramfunc)
                0x00000000                _ramfunc_length = SIZEOF (.ramfunc)
                0x00002000                _bmxdkpba_address = (_ramfunc_begin - 0xa0000000)
                0x00008000                _bmxdudba_address = 0x8000
                0x00008000                _bmxdupba_address = 0x8000
                0xa0008000                _stack = (_ramfunc_length > 0x0)?(_ramfunc_begin - 0x4):0xa0008000
                0x00000001                ASSERT (((_min_stack_size + _min_heap_size) <= (_stack - _heap)), Not enough space to allocate both stack and heap.  Reduce heap and/or stack size.)

.pdr            0x00000000      0xbe0
 *(.pdr)
 .pdr           0x00000000       0xa0 C:/Program Files/Microchip/MPLAB C32/bin/../lib/gcc/pic32mx/3.4.4/../../../../pic32mx/lib/size/crt0.o
 .pdr           0x000000a0       0x20 Objects - Graphics Primitives Layer Demo\MainDemo.o
 .pdr           0x000000c0      0x1c0 Objects - Graphics Primitives Layer Demo\Primitive.o
 .pdr           0x00000280      0x3a0 Objects - Graphics Primitives Layer Demo\DisplayDriver.o
 .pdr           0x00000620       0x20 C:/Program Files/Microchip/MPLAB C32/bin/../lib/gcc/pic32mx/3.4.4/../../../../pic32mx/lib/size\libc.a(memcpy.o)
 .pdr           0x00000640       0x20 C:/Program Files/Microchip/MPLAB C32/bin/../lib/gcc/pic32mx/3.4.4/../../../../pic32mx/lib/size\libc.a(general-exception.o)
 .pdr           0x00000660       0x20 C:/Program Files/Microchip/MPLAB C32/bin/../lib/gcc/pic32mx/3.4.4/../../../../pic32mx/lib/size\libc.a(exit.o)
 .pdr           0x00000680       0xa0 C:/Program Files/Microchip/MPLAB C32/bin/../lib/gcc/pic32mx/3.4.4/../../../../pic32mx/lib/size\libc.a(_iobfuncs.o)
 .pdr           0x00000720      0x2c0 C:/Program Files/Microchip/MPLAB C32/bin/../lib/gcc/pic32mx/3.4.4/../../../../pic32mx/lib/size\libc.a(stubs.o)
 .pdr           0x000009e0       0x20 C:/Program Files/Microchip/MPLAB C32/bin/../lib/gcc/pic32mx/3.4.4/../../../../pic32mx/lib/size\libc.a(default-general-exception-handler.o)
 .pdr           0x00000a00       0x20 C:/Program Files/Microchip/MPLAB C32/bin/../lib/gcc/pic32mx/3.4.4/../../../../pic32mx/lib/size\libc.a(default-bootstrap-exception-handler.o)
 .pdr           0x00000a20       0x20 C:/Program Files/Microchip/MPLAB C32/bin/../lib/gcc/pic32mx/3.4.4/../../../../pic32mx/lib/size\libc.a(default-on-reset.o)
 .pdr           0x00000a40       0x20 C:/Program Files/Microchip/MPLAB C32/bin/../lib/gcc/pic32mx/3.4.4/../../../../pic32mx/lib/size\libc.a(default-on-bootstrap.o)
 .pdr           0x00000a60       0x20 C:/Program Files/Microchip/MPLAB C32/bin/../lib/gcc/pic32mx/3.4.4/../../../../pic32mx/lib/size\libc.a(default-nmi-handler.o)
 .pdr           0x00000a80       0x20 C:/Program Files/Microchip/MPLAB C32/bin/../lib/gcc/pic32mx/3.4.4/../../../../pic32mx/lib/size\libc.a(_mon_getc.o)
 .pdr           0x00000aa0       0x20 C:/Program Files/Microchip/MPLAB C32/bin/../lib/gcc/pic32mx/3.4.4/../../../../pic32mx/lib/size\libc.a(_mon_write.o)
 .pdr           0x00000ac0       0x20 C:/Program Files/Microchip/MPLAB C32/bin/../lib/gcc/pic32mx/3.4.4/../../../../pic32mx/lib/size\libc.a(_exit.o)
 .pdr           0x00000ae0       0x20 C:/Program Files/Microchip/MPLAB C32/bin/../lib/gcc/pic32mx/3.4.4/../../../../pic32mx/lib/size\libc.a(_mon_putc.o)
 .pdr           0x00000b00       0x20 C:/Program Files/Microchip/MPLAB C32/bin/../lib/gcc/pic32mx/3.4.4/../../../../pic32mx/lib/size\libmchp_peripheral.a(int_disable_interrupts_lib.o)
 .pdr           0x00000b20       0x20 C:/Program Files/Microchip/MPLAB C32/bin/../lib/gcc/pic32mx/3.4.4/../../../../pic32mx/lib/size\libmchp_peripheral.a(int_enable_mv_int_lib.o)
 .pdr           0x00000b40       0x20 C:/Program Files/Microchip/MPLAB C32/bin/../lib/gcc/pic32mx/3.4.4/../../../../pic32mx/lib/size\libmchp_peripheral.a(int_restore_interrupts_lib.o)
 .pdr           0x00000b60       0x20 C:/Program Files/Microchip/MPLAB C32/bin/../lib/gcc/pic32mx/3.4.4/../../../../pic32mx/lib/size\libmchp_peripheral.a(open_core_timer_lib.o)
 .pdr           0x00000b80       0x40 C:/Program Files/Microchip/MPLAB C32/bin/../lib/gcc/pic32mx/3.4.4/../../../../pic32mx/lib/size\libmchp_peripheral.a(pcache.o)
 .pdr           0x00000bc0       0x20 C:/Program Files/Microchip/MPLAB C32/bin/../lib/gcc/pic32mx/3.4.4/../../../../pic32mx/lib/size\libmchp_peripheral.a(int_enable_interrupts_lib.o)

.reginfo        0x00000000       0x18
 *(.reginfo)
 .reginfo       0x00000000       0x18 C:/Program Files/Microchip/MPLAB C32/bin/../lib/gcc/pic32mx/3.4.4/../../../../pic32mx/lib/size/crt0.o

.stab
 *(.stab)

.stabstr
 *(.stabstr)

.stab.excl
 *(.stab.excl)

.stab.exclstr
 *(.stab.exclstr)

.stab.index
 *(.stab.index)

.stab.indexstr
 *(.stab.indexstr)

.comment        0x00000000      0x8c5
 *(.comment)
 .comment       0x00000000       0x2d Objects - Graphics Primitives Layer Demo\MainDemo.o
 .comment       0x0000002d       0x2d Objects - Graphics Primitives Layer Demo\Pictures PIC32.o
 .comment       0x0000005a       0x2d Objects - Graphics Primitives Layer Demo\Font25PixelsHeight.o
 .comment       0x00000087       0x2d Objects - Graphics Primitives Layer Demo\Window.o
 .comment       0x000000b4       0x2d Objects - Graphics Primitives Layer Demo\Button.o
 .comment       0x000000e1       0x2d Objects - Graphics Primitives Layer Demo\Chart.o
 .comment       0x0000010e       0x2d Objects - Graphics Primitives Layer Demo\CheckBox.o
 .comment       0x0000013b       0x2d Objects - Graphics Primitives Layer Demo\EditBox.o
 .comment       0x00000168       0x2d Objects - Graphics Primitives Layer Demo\GOL.o
 .comment       0x00000195       0x2d Objects - Graphics Primitives Layer Demo\GOLFontDefault.o
 .comment       0x000001c2       0x2d Objects - Graphics Primitives Layer Demo\Grid.o
 .comment       0x000001ef       0x2d Objects - Graphics Primitives Layer Demo\GroupBox.o
 .comment       0x0000021c       0x2d Objects - Graphics Primitives Layer Demo\ListBox.o
 .comment       0x00000249       0x2d Objects - Graphics Primitives Layer Demo\Meter.o
 .comment       0x00000276       0x2d Objects - Graphics Primitives Layer Demo\Picture.o
 .comment       0x000002a3       0x2d Objects - Graphics Primitives Layer Demo\Primitive.o
 .comment       0x000002d0       0x2d Objects - Graphics Primitives Layer Demo\ProgressBar.o
 .comment       0x000002fd       0x2d Objects - Graphics Primitives Layer Demo\RadioButton.o
 .comment       0x0000032a       0x2d Objects - Graphics Primitives Layer Demo\RoundDial.o
 .comment       0x00000357       0x2d Objects - Graphics Primitives Layer Demo\Slider.o
 .comment       0x00000384       0x2d Objects - Graphics Primitives Layer Demo\StaticText.o
 .comment       0x000003b1       0x2d Objects - Graphics Primitives Layer Demo\DisplayDriver.o
 .comment       0x000003de       0x7a C:/Program Files/Microchip/MPLAB C32/bin/../lib/gcc/pic32mx/3.4.4/../../../../pic32mx/lib/size\libc.a(exit.o)
 .comment       0x00000458       0x80 C:/Program Files/Microchip/MPLAB C32/bin/../lib/gcc/pic32mx/3.4.4/../../../../pic32mx/lib/size\libc.a(_iobdata.o)
 .comment       0x000004d8       0x81 C:/Program Files/Microchip/MPLAB C32/bin/../lib/gcc/pic32mx/3.4.4/../../../../pic32mx/lib/size\libc.a(_iobfuncs.o)
 .comment       0x00000559       0x7b C:/Program Files/Microchip/MPLAB C32/bin/../lib/gcc/pic32mx/3.4.4/../../../../pic32mx/lib/size\libc.a(stubs.o)
 .comment       0x000005d4       0x2d C:/Program Files/Microchip/MPLAB C32/bin/../lib/gcc/pic32mx/3.4.4/../../../../pic32mx/lib/size\libc.a(default-general-exception-handler.o)
 .comment       0x00000601       0x2d C:/Program Files/Microchip/MPLAB C32/bin/../lib/gcc/pic32mx/3.4.4/../../../../pic32mx/lib/size\libc.a(default-bootstrap-exception-handler.o)
 .comment       0x0000062e       0x2d C:/Program Files/Microchip/MPLAB C32/bin/../lib/gcc/pic32mx/3.4.4/../../../../pic32mx/lib/size\libc.a(default-on-reset.o)
 .comment       0x0000065b       0x2d C:/Program Files/Microchip/MPLAB C32/bin/../lib/gcc/pic32mx/3.4.4/../../../../pic32mx/lib/size\libc.a(default-on-bootstrap.o)
 .comment       0x00000688       0x2d C:/Program Files/Microchip/MPLAB C32/bin/../lib/gcc/pic32mx/3.4.4/../../../../pic32mx/lib/size\libc.a(_mon_getc.o)
 .comment       0x000006b5       0x2d C:/Program Files/Microchip/MPLAB C32/bin/../lib/gcc/pic32mx/3.4.4/../../../../pic32mx/lib/size\libc.a(_mon_write.o)
 .comment       0x000006e2       0x2d C:/Program Files/Microchip/MPLAB C32/bin/../lib/gcc/pic32mx/3.4.4/../../../../pic32mx/lib/size\libc.a(_exit.o)
 .comment       0x0000070f       0x7b C:/Program Files/Microchip/MPLAB C32/bin/../lib/gcc/pic32mx/3.4.4/../../../../pic32mx/lib/size\libc.a(errno.o)
 .comment       0x0000078a       0x2d C:/Program Files/Microchip/MPLAB C32/bin/../lib/gcc/pic32mx/3.4.4/../../../../pic32mx/lib/size\libc.a(_mon_putc.o)
 .comment       0x000007b7       0x2d C:/Program Files/Microchip/MPLAB C32/bin/../lib/gcc/pic32mx/3.4.4/../../../../pic32mx/lib/size\libmchp_peripheral.a(int_disable_interrupts_lib.o)
 .comment       0x000007e4       0x2d C:/Program Files/Microchip/MPLAB C32/bin/../lib/gcc/pic32mx/3.4.4/../../../../pic32mx/lib/size\libmchp_peripheral.a(int_enable_mv_int_lib.o)
 .comment       0x00000811       0x2d C:/Program Files/Microchip/MPLAB C32/bin/../lib/gcc/pic32mx/3.4.4/../../../../pic32mx/lib/size\libmchp_peripheral.a(int_restore_interrupts_lib.o)
 .comment       0x0000083e       0x2d C:/Program Files/Microchip/MPLAB C32/bin/../lib/gcc/pic32mx/3.4.4/../../../../pic32mx/lib/size\libmchp_peripheral.a(open_core_timer_lib.o)
 .comment       0x0000086b       0x2d C:/Program Files/Microchip/MPLAB C32/bin/../lib/gcc/pic32mx/3.4.4/../../../../pic32mx/lib/size\libmchp_peripheral.a(pcache.o)
 .comment       0x00000898       0x2d C:/Program Files/Microchip/MPLAB C32/bin/../lib/gcc/pic32mx/3.4.4/../../../../pic32mx/lib/size\libmchp_peripheral.a(int_enable_interrupts_lib.o)

.debug
 *(.debug)

.line
 *(.line)

.debug_srcinfo
 *(.debug_srcinfo)

.debug_sfnames
 *(.debug_sfnames)

.debug_aranges  0x00000000      0x478
 *(.debug_aranges)
 .debug_aranges
                0x00000000       0x40 C:/Program Files/Microchip/MPLAB C32/bin/../lib/gcc/pic32mx/3.4.4/../../../../pic32mx/lib/size/crt0.o
 .debug_aranges
                0x00000040       0x20 Objects - Graphics Primitives Layer Demo\MainDemo.o
 .debug_aranges
                0x00000060       0x20 Objects - Graphics Primitives Layer Demo\Primitive.o
 .debug_aranges
                0x00000080       0x20 Objects - Graphics Primitives Layer Demo\DisplayDriver.o
 .debug_aranges
                0x000000a0       0x20 C:/Program Files/Microchip/MPLAB C32/bin/../lib/gcc/pic32mx/3.4.4/../../../../pic32mx/lib/size\libc.a(memcpy.o)
 .debug_aranges
                0x000000c0       0x20 C:/Program Files/Microchip/MPLAB C32/bin/../lib/gcc/pic32mx/3.4.4/../../../../pic32mx/lib/size\libc.a(general-exception.o)
 .debug_aranges
                0x000000e0       0x28 C:/Program Files/Microchip/MPLAB C32/bin/../lib/gcc/pic32mx/3.4.4/../../../../pic32mx/lib/size\libc.a(exit.o)
 .debug_aranges
                0x00000108       0x48 C:/Program Files/Microchip/MPLAB C32/bin/../lib/gcc/pic32mx/3.4.4/../../../../pic32mx/lib/size\libc.a(_iobfuncs.o)
 .debug_aranges
                0x00000150       0xd0 C:/Program Files/Microchip/MPLAB C32/bin/../lib/gcc/pic32mx/3.4.4/../../../../pic32mx/lib/size\libc.a(stubs.o)
 .debug_aranges
                0x00000220       0x28 C:/Program Files/Microchip/MPLAB C32/bin/../lib/gcc/pic32mx/3.4.4/../../../../pic32mx/lib/size\libc.a(default-general-exception-handler.o)
 .debug_aranges
                0x00000248       0x28 C:/Program Files/Microchip/MPLAB C32/bin/../lib/gcc/pic32mx/3.4.4/../../../../pic32mx/lib/size\libc.a(default-bootstrap-exception-handler.o)
 .debug_aranges
                0x00000270       0x28 C:/Program Files/Microchip/MPLAB C32/bin/../lib/gcc/pic32mx/3.4.4/../../../../pic32mx/lib/size\libc.a(default-on-reset.o)
 .debug_aranges
                0x00000298       0x28 C:/Program Files/Microchip/MPLAB C32/bin/../lib/gcc/pic32mx/3.4.4/../../../../pic32mx/lib/size\libc.a(default-on-bootstrap.o)
 .debug_aranges
                0x000002c0       0x20 C:/Program Files/Microchip/MPLAB C32/bin/../lib/gcc/pic32mx/3.4.4/../../../../pic32mx/lib/size\libc.a(default-nmi-handler.o)
 .debug_aranges
                0x000002e0       0x28 C:/Program Files/Microchip/MPLAB C32/bin/../lib/gcc/pic32mx/3.4.4/../../../../pic32mx/lib/size\libc.a(_mon_getc.o)
 .debug_aranges
                0x00000308       0x28 C:/Program Files/Microchip/MPLAB C32/bin/../lib/gcc/pic32mx/3.4.4/../../../../pic32mx/lib/size\libc.a(_mon_write.o)
 .debug_aranges
                0x00000330       0x28 C:/Program Files/Microchip/MPLAB C32/bin/../lib/gcc/pic32mx/3.4.4/../../../../pic32mx/lib/size\libc.a(_exit.o)
 .debug_aranges
                0x00000358       0x28 C:/Program Files/Microchip/MPLAB C32/bin/../lib/gcc/pic32mx/3.4.4/../../../../pic32mx/lib/size\libc.a(_mon_putc.o)
 .debug_aranges
                0x00000380       0x28 C:/Program Files/Microchip/MPLAB C32/bin/../lib/gcc/pic32mx/3.4.4/../../../../pic32mx/lib/size\libmchp_peripheral.a(int_disable_interrupts_lib.o)
 .debug_aranges
                0x000003a8       0x28 C:/Program Files/Microchip/MPLAB C32/bin/../lib/gcc/pic32mx/3.4.4/../../../../pic32mx/lib/size\libmchp_peripheral.a(int_enable_mv_int_lib.o)
 .debug_aranges
                0x000003d0       0x28 C:/Program Files/Microchip/MPLAB C32/bin/../lib/gcc/pic32mx/3.4.4/../../../../pic32mx/lib/size\libmchp_peripheral.a(int_restore_interrupts_lib.o)
 .debug_aranges
                0x000003f8       0x28 C:/Program Files/Microchip/MPLAB C32/bin/../lib/gcc/pic32mx/3.4.4/../../../../pic32mx/lib/size\libmchp_peripheral.a(open_core_timer_lib.o)
 .debug_aranges
                0x00000420       0x30 C:/Program Files/Microchip/MPLAB C32/bin/../lib/gcc/pic32mx/3.4.4/../../../../pic32mx/lib/size\libmchp_peripheral.a(pcache.o)
 .debug_aranges
                0x00000450       0x28 C:/Program Files/Microchip/MPLAB C32/bin/../lib/gcc/pic32mx/3.4.4/../../../../pic32mx/lib/size\libmchp_peripheral.a(int_enable_interrupts_lib.o)

.debug_pubnames
                0x00000000      0xa17
 *(.debug_pubnames)
 .debug_pubnames
                0x00000000       0x1b Objects - Graphics Primitives Layer Demo\MainDemo.o
 .debug_pubnames
                0x0000001b       0x7b Objects - Graphics Primitives Layer Demo\Pictures PIC32.o
 .debug_pubnames
                0x00000096       0x25 Objects - Graphics Primitives Layer Demo\Font25PixelsHeight.o
 .debug_pubnames
                0x000000bb      0x15f Objects - Graphics Primitives Layer Demo\Primitive.o
 .debug_pubnames
                0x0000021a      0x25e Objects - Graphics Primitives Layer Demo\DisplayDriver.o
 .debug_pubnames
                0x00000478       0x1b C:/Program Files/Microchip/MPLAB C32/bin/../lib/gcc/pic32mx/3.4.4/../../../../pic32mx/lib/size\libc.a(exit.o)
 .debug_pubnames
                0x00000493       0x70 C:/Program Files/Microchip/MPLAB C32/bin/../lib/gcc/pic32mx/3.4.4/../../../../pic32mx/lib/size\libc.a(_iobfuncs.o)
 .debug_pubnames
                0x00000503      0x2da C:/Program Files/Microchip/MPLAB C32/bin/../lib/gcc/pic32mx/3.4.4/../../../../pic32mx/lib/size\libc.a(stubs.o)
 .debug_pubnames
                0x000007dd       0x31 C:/Program Files/Microchip/MPLAB C32/bin/../lib/gcc/pic32mx/3.4.4/../../../../pic32mx/lib/size\libc.a(default-general-exception-handler.o)
 .debug_pubnames
                0x0000080e       0x33 C:/Program Files/Microchip/MPLAB C32/bin/../lib/gcc/pic32mx/3.4.4/../../../../pic32mx/lib/size\libc.a(default-bootstrap-exception-handler.o)
 .debug_pubnames
                0x00000841       0x20 C:/Program Files/Microchip/MPLAB C32/bin/../lib/gcc/pic32mx/3.4.4/../../../../pic32mx/lib/size\libc.a(default-on-reset.o)
 .debug_pubnames
                0x00000861       0x24 C:/Program Files/Microchip/MPLAB C32/bin/../lib/gcc/pic32mx/3.4.4/../../../../pic32mx/lib/size\libc.a(default-on-bootstrap.o)
 .debug_pubnames
                0x00000885       0x20 C:/Program Files/Microchip/MPLAB C32/bin/../lib/gcc/pic32mx/3.4.4/../../../../pic32mx/lib/size\libc.a(_mon_getc.o)
 .debug_pubnames
                0x000008a5       0x21 C:/Program Files/Microchip/MPLAB C32/bin/../lib/gcc/pic32mx/3.4.4/../../../../pic32mx/lib/size\libc.a(_mon_write.o)
 .debug_pubnames
                0x000008c6       0x1c C:/Program Files/Microchip/MPLAB C32/bin/../lib/gcc/pic32mx/3.4.4/../../../../pic32mx/lib/size\libc.a(_exit.o)
 .debug_pubnames
                0x000008e2       0x20 C:/Program Files/Microchip/MPLAB C32/bin/../lib/gcc/pic32mx/3.4.4/../../../../pic32mx/lib/size\libc.a(_mon_putc.o)
 .debug_pubnames
                0x00000902       0x2b C:/Program Files/Microchip/MPLAB C32/bin/../lib/gcc/pic32mx/3.4.4/../../../../pic32mx/lib/size\libmchp_peripheral.a(int_disable_interrupts_lib.o)
 .debug_pubnames
                0x0000092d       0x36 C:/Program Files/Microchip/MPLAB C32/bin/../lib/gcc/pic32mx/3.4.4/../../../../pic32mx/lib/size\libmchp_peripheral.a(int_enable_mv_int_lib.o)
 .debug_pubnames
                0x00000963       0x2b C:/Program Files/Microchip/MPLAB C32/bin/../lib/gcc/pic32mx/3.4.4/../../../../pic32mx/lib/size\libmchp_peripheral.a(int_restore_interrupts_lib.o)
 .debug_pubnames
                0x0000098e       0x24 C:/Program Files/Microchip/MPLAB C32/bin/../lib/gcc/pic32mx/3.4.4/../../../../pic32mx/lib/size\libmchp_peripheral.a(open_core_timer_lib.o)
 .debug_pubnames
                0x000009b2       0x3b C:/Program Files/Microchip/MPLAB C32/bin/../lib/gcc/pic32mx/3.4.4/../../../../pic32mx/lib/size\libmchp_peripheral.a(pcache.o)
 .debug_pubnames
                0x000009ed       0x2a C:/Program Files/Microchip/MPLAB C32/bin/../lib/gcc/pic32mx/3.4.4/../../../../pic32mx/lib/size\libmchp_peripheral.a(int_enable_interrupts_lib.o)

.debug_info     0x00000000     0x5407
 *(.debug_info .gnu.linkonce.wi.*)
 .debug_info    0x00000000       0xdd C:/Program Files/Microchip/MPLAB C32/bin/../lib/gcc/pic32mx/3.4.4/../../../../pic32mx/lib/size/crt0.o
 .debug_info    0x000000dd      0x5a2 Objects - Graphics Primitives Layer Demo\MainDemo.o
 .debug_info    0x0000067f      0x372 Objects - Graphics Primitives Layer Demo\Pictures PIC32.o
 .debug_info    0x000009f1       0xaa Objects - Graphics Primitives Layer Demo\Font25PixelsHeight.o
 .debug_info    0x00000a9b      0x20e Objects - Graphics Primitives Layer Demo\Window.o
 .debug_info    0x00000ca9      0x20e Objects - Graphics Primitives Layer Demo\Button.o
 .debug_info    0x00000eb7      0x20e Objects - Graphics Primitives Layer Demo\Chart.o
 .debug_info    0x000010c5      0x20e Objects - Graphics Primitives Layer Demo\CheckBox.o
 .debug_info    0x000012d3      0x20e Objects - Graphics Primitives Layer Demo\EditBox.o
 .debug_info    0x000014e1      0x20e Objects - Graphics Primitives Layer Demo\GOL.o
 .debug_info    0x000016ef      0x20e Objects - Graphics Primitives Layer Demo\Grid.o
 .debug_info    0x000018fd      0x20e Objects - Graphics Primitives Layer Demo\GroupBox.o
 .debug_info    0x00001b0b      0x20e Objects - Graphics Primitives Layer Demo\ListBox.o
 .debug_info    0x00001d19      0x20e Objects - Graphics Primitives Layer Demo\Meter.o
 .debug_info    0x00001f27      0x20e Objects - Graphics Primitives Layer Demo\Picture.o
 .debug_info    0x00002135     0x1096 Objects - Graphics Primitives Layer Demo\Primitive.o
 .debug_info    0x000031cb      0x20e Objects - Graphics Primitives Layer Demo\ProgressBar.o
 .debug_info    0x000033d9      0x20e Objects - Graphics Primitives Layer Demo\RadioButton.o
 .debug_info    0x000035e7      0x20e Objects - Graphics Primitives Layer Demo\RoundDial.o
 .debug_info    0x000037f5      0x20e Objects - Graphics Primitives Layer Demo\Slider.o
 .debug_info    0x00003a03      0x20e Objects - Graphics Primitives Layer Demo\StaticText.o
 .debug_info    0x00003c11     0x1025 Objects - Graphics Primitives Layer Demo\DisplayDriver.o
 .debug_info    0x00004c36       0xe9 C:/Program Files/Microchip/MPLAB C32/bin/../lib/gcc/pic32mx/3.4.4/../../../../pic32mx/lib/size\libc.a(memcpy.o)
 .debug_info    0x00004d1f       0xf2 C:/Program Files/Microchip/MPLAB C32/bin/../lib/gcc/pic32mx/3.4.4/../../../../pic32mx/lib/size\libc.a(general-exception.o)
 .debug_info    0x00004e11       0x30 C:/Program Files/Microchip/MPLAB C32/bin/../lib/gcc/pic32mx/3.4.4/../../../../pic32mx/lib/size\libc.a(exit.o)
 .debug_info    0x00004e41       0x78 C:/Program Files/Microchip/MPLAB C32/bin/../lib/gcc/pic32mx/3.4.4/../../../../pic32mx/lib/size\libc.a(_iobfuncs.o)
 .debug_info    0x00004eb9      0x1aa C:/Program Files/Microchip/MPLAB C32/bin/../lib/gcc/pic32mx/3.4.4/../../../../pic32mx/lib/size\libc.a(stubs.o)
 .debug_info    0x00005063       0x30 C:/Program Files/Microchip/MPLAB C32/bin/../lib/gcc/pic32mx/3.4.4/../../../../pic32mx/lib/size\libc.a(default-general-exception-handler.o)
 .debug_info    0x00005093       0x30 C:/Program Files/Microchip/MPLAB C32/bin/../lib/gcc/pic32mx/3.4.4/../../../../pic32mx/lib/size\libc.a(default-bootstrap-exception-handler.o)
 .debug_info    0x000050c3       0x30 C:/Program Files/Microchip/MPLAB C32/bin/../lib/gcc/pic32mx/3.4.4/../../../../pic32mx/lib/size\libc.a(default-on-reset.o)
 .debug_info    0x000050f3       0x30 C:/Program Files/Microchip/MPLAB C32/bin/../lib/gcc/pic32mx/3.4.4/../../../../pic32mx/lib/size\libc.a(default-on-bootstrap.o)
 .debug_info    0x00005123       0xf2 C:/Program Files/Microchip/MPLAB C32/bin/../lib/gcc/pic32mx/3.4.4/../../../../pic32mx/lib/size\libc.a(default-nmi-handler.o)
 .debug_info    0x00005215       0x30 C:/Program Files/Microchip/MPLAB C32/bin/../lib/gcc/pic32mx/3.4.4/../../../../pic32mx/lib/size\libc.a(_mon_getc.o)
 .debug_info    0x00005245       0x30 C:/Program Files/Microchip/MPLAB C32/bin/../lib/gcc/pic32mx/3.4.4/../../../../pic32mx/lib/size\libc.a(_mon_write.o)
 .debug_info    0x00005275       0x30 C:/Program Files/Microchip/MPLAB C32/bin/../lib/gcc/pic32mx/3.4.4/../../../../pic32mx/lib/size\libc.a(_exit.o)
 .debug_info    0x000052a5       0x30 C:/Program Files/Microchip/MPLAB C32/bin/../lib/gcc/pic32mx/3.4.4/../../../../pic32mx/lib/size\libc.a(_mon_putc.o)
 .debug_info    0x000052d5       0x30 C:/Program Files/Microchip/MPLAB C32/bin/../lib/gcc/pic32mx/3.4.4/../../../../pic32mx/lib/size\libmchp_peripheral.a(int_disable_interrupts_lib.o)
 .debug_info    0x00005305       0x30 C:/Program Files/Microchip/MPLAB C32/bin/../lib/gcc/pic32mx/3.4.4/../../../../pic32mx/lib/size\libmchp_peripheral.a(int_enable_mv_int_lib.o)
 .debug_info    0x00005335       0x30 C:/Program Files/Microchip/MPLAB C32/bin/../lib/gcc/pic32mx/3.4.4/../../../../pic32mx/lib/size\libmchp_peripheral.a(int_restore_interrupts_lib.o)
 .debug_info    0x00005365       0x30 C:/Program Files/Microchip/MPLAB C32/bin/../lib/gcc/pic32mx/3.4.4/../../../../pic32mx/lib/size\libmchp_peripheral.a(open_core_timer_lib.o)
 .debug_info    0x00005395       0x42 C:/Program Files/Microchip/MPLAB C32/bin/../lib/gcc/pic32mx/3.4.4/../../../../pic32mx/lib/size\libmchp_peripheral.a(pcache.o)
 .debug_info    0x000053d7       0x30 C:/Program Files/Microchip/MPLAB C32/bin/../lib/gcc/pic32mx/3.4.4/../../../../pic32mx/lib/size\libmchp_peripheral.a(int_enable_interrupts_lib.o)

.debug_abbrev   0x00000000     0x1552
 *(.debug_abbrev)
 .debug_abbrev  0x00000000       0x10 C:/Program Files/Microchip/MPLAB C32/bin/../lib/gcc/pic32mx/3.4.4/../../../../pic32mx/lib/size/crt0.o
 .debug_abbrev  0x00000010      0x1f7 Objects - Graphics Primitives Layer Demo\MainDemo.o
 .debug_abbrev  0x00000207      0x121 Objects - Graphics Primitives Layer Demo\Pictures PIC32.o
 .debug_abbrev  0x00000328       0x7f Objects - Graphics Primitives Layer Demo\Font25PixelsHeight.o
 .debug_abbrev  0x000003a7       0xab Objects - Graphics Primitives Layer Demo\Window.o
 .debug_abbrev  0x00000452       0xab Objects - Graphics Primitives Layer Demo\Button.o
 .debug_abbrev  0x000004fd       0xab Objects - Graphics Primitives Layer Demo\Chart.o
 .debug_abbrev  0x000005a8       0xab Objects - Graphics Primitives Layer Demo\CheckBox.o
 .debug_abbrev  0x00000653       0xab Objects - Graphics Primitives Layer Demo\EditBox.o
 .debug_abbrev  0x000006fe       0xab Objects - Graphics Primitives Layer Demo\GOL.o
 .debug_abbrev  0x000007a9        0x1 Objects - Graphics Primitives Layer Demo\GOLFontDefault.o
 .debug_abbrev  0x000007aa       0xab Objects - Graphics Primitives Layer Demo\Grid.o
 .debug_abbrev  0x00000855       0xab Objects - Graphics Primitives Layer Demo\GroupBox.o
 .debug_abbrev  0x00000900       0xab Objects - Graphics Primitives Layer Demo\ListBox.o
 .debug_abbrev  0x000009ab       0xab Objects - Graphics Primitives Layer Demo\Meter.o
 .debug_abbrev  0x00000a56       0xab Objects - Graphics Primitives Layer Demo\Picture.o
 .debug_abbrev  0x00000b01      0x22f Objects - Graphics Primitives Layer Demo\Primitive.o
 .debug_abbrev  0x00000d30       0xab Objects - Graphics Primitives Layer Demo\ProgressBar.o
 .debug_abbrev  0x00000ddb       0xab Objects - Graphics Primitives Layer Demo\RadioButton.o
 .debug_abbrev  0x00000e86       0xab Objects - Graphics Primitives Layer Demo\RoundDial.o
 .debug_abbrev  0x00000f31       0xab Objects - Graphics Primitives Layer Demo\Slider.o
 .debug_abbrev  0x00000fdc       0xab Objects - Graphics Primitives Layer Demo\StaticText.o
 .debug_abbrev  0x00001087      0x23a Objects - Graphics Primitives Layer Demo\DisplayDriver.o
 .debug_abbrev  0x000012c1       0x14 C:/Program Files/Microchip/MPLAB C32/bin/../lib/gcc/pic32mx/3.4.4/../../../../pic32mx/lib/size\libc.a(memcpy.o)
 .debug_abbrev  0x000012d5       0x14 C:/Program Files/Microchip/MPLAB C32/bin/../lib/gcc/pic32mx/3.4.4/../../../../pic32mx/lib/size\libc.a(general-exception.o)
 .debug_abbrev  0x000012e9       0x23 C:/Program Files/Microchip/MPLAB C32/bin/../lib/gcc/pic32mx/3.4.4/../../../../pic32mx/lib/size\libc.a(exit.o)
 .debug_abbrev  0x0000130c        0x1 C:/Program Files/Microchip/MPLAB C32/bin/../lib/gcc/pic32mx/3.4.4/../../../../pic32mx/lib/size\libc.a(_iobdata.o)
 .debug_abbrev  0x0000130d       0x23 C:/Program Files/Microchip/MPLAB C32/bin/../lib/gcc/pic32mx/3.4.4/../../../../pic32mx/lib/size\libc.a(_iobfuncs.o)
 .debug_abbrev  0x00001330       0x23 C:/Program Files/Microchip/MPLAB C32/bin/../lib/gcc/pic32mx/3.4.4/../../../../pic32mx/lib/size\libc.a(stubs.o)
 .debug_abbrev  0x00001353       0x23 C:/Program Files/Microchip/MPLAB C32/bin/../lib/gcc/pic32mx/3.4.4/../../../../pic32mx/lib/size\libc.a(default-general-exception-handler.o)
 .debug_abbrev  0x00001376       0x23 C:/Program Files/Microchip/MPLAB C32/bin/../lib/gcc/pic32mx/3.4.4/../../../../pic32mx/lib/size\libc.a(default-bootstrap-exception-handler.o)
 .debug_abbrev  0x00001399       0x23 C:/Program Files/Microchip/MPLAB C32/bin/../lib/gcc/pic32mx/3.4.4/../../../../pic32mx/lib/size\libc.a(default-on-reset.o)
 .debug_abbrev  0x000013bc       0x23 C:/Program Files/Microchip/MPLAB C32/bin/../lib/gcc/pic32mx/3.4.4/../../../../pic32mx/lib/size\libc.a(default-on-bootstrap.o)
 .debug_abbrev  0x000013df       0x14 C:/Program Files/Microchip/MPLAB C32/bin/../lib/gcc/pic32mx/3.4.4/../../../../pic32mx/lib/size\libc.a(default-nmi-handler.o)
 .debug_abbrev  0x000013f3       0x23 C:/Program Files/Microchip/MPLAB C32/bin/../lib/gcc/pic32mx/3.4.4/../../../../pic32mx/lib/size\libc.a(_mon_getc.o)
 .debug_abbrev  0x00001416       0x23 C:/Program Files/Microchip/MPLAB C32/bin/../lib/gcc/pic32mx/3.4.4/../../../../pic32mx/lib/size\libc.a(_mon_write.o)
 .debug_abbrev  0x00001439       0x23 C:/Program Files/Microchip/MPLAB C32/bin/../lib/gcc/pic32mx/3.4.4/../../../../pic32mx/lib/size\libc.a(_exit.o)
 .debug_abbrev  0x0000145c        0x1 C:/Program Files/Microchip/MPLAB C32/bin/../lib/gcc/pic32mx/3.4.4/../../../../pic32mx/lib/size\libc.a(errno.o)
 .debug_abbrev  0x0000145d       0x23 C:/Program Files/Microchip/MPLAB C32/bin/../lib/gcc/pic32mx/3.4.4/../../../../pic32mx/lib/size\libc.a(_mon_putc.o)
 .debug_abbrev  0x00001480       0x23 C:/Program Files/Microchip/MPLAB C32/bin/../lib/gcc/pic32mx/3.4.4/../../../../pic32mx/lib/size\libmchp_peripheral.a(int_disable_interrupts_lib.o)
 .debug_abbrev  0x000014a3       0x23 C:/Program Files/Microchip/MPLAB C32/bin/../lib/gcc/pic32mx/3.4.4/../../../../pic32mx/lib/size\libmchp_peripheral.a(int_enable_mv_int_lib.o)
 .debug_abbrev  0x000014c6       0x23 C:/Program Files/Microchip/MPLAB C32/bin/../lib/gcc/pic32mx/3.4.4/../../../../pic32mx/lib/size\libmchp_peripheral.a(int_restore_interrupts_lib.o)
 .debug_abbrev  0x000014e9       0x23 C:/Program Files/Microchip/MPLAB C32/bin/../lib/gcc/pic32mx/3.4.4/../../../../pic32mx/lib/size\libmchp_peripheral.a(open_core_timer_lib.o)
 .debug_abbrev  0x0000150c       0x23 C:/Program Files/Microchip/MPLAB C32/bin/../lib/gcc/pic32mx/3.4.4/../../../../pic32mx/lib/size\libmchp_peripheral.a(pcache.o)
 .debug_abbrev  0x0000152f       0x23 C:/Program Files/Microchip/MPLAB C32/bin/../lib/gcc/pic32mx/3.4.4/../../../../pic32mx/lib/size\libmchp_peripheral.a(int_enable_interrupts_lib.o)

.debug_line     0x00000000     0x228a
 *(.debug_line)
 .debug_line    0x00000000      0x137 C:/Program Files/Microchip/MPLAB C32/bin/../lib/gcc/pic32mx/3.4.4/../../../../pic32mx/lib/size/crt0.o
 .debug_line    0x00000137      0x2d3 Objects - Graphics Primitives Layer Demo\MainDemo.o
 .debug_line    0x0000040a       0xfc Objects - Graphics Primitives Layer Demo\Pictures PIC32.o
 .debug_line    0x00000506       0x32 Objects - Graphics Primitives Layer Demo\Font25PixelsHeight.o
 .debug_line    0x00000538       0x90 Objects - Graphics Primitives Layer Demo\Window.o
 .debug_line    0x000005c8       0x90 Objects - Graphics Primitives Layer Demo\Button.o
 .debug_line    0x00000658       0x90 Objects - Graphics Primitives Layer Demo\Chart.o
 .debug_line    0x000006e8       0x90 Objects - Graphics Primitives Layer Demo\CheckBox.o
 .debug_line    0x00000778       0x90 Objects - Graphics Primitives Layer Demo\EditBox.o
 .debug_line    0x00000808       0x90 Objects - Graphics Primitives Layer Demo\GOL.o
 .debug_line    0x00000898       0x90 Objects - Graphics Primitives Layer Demo\Grid.o
 .debug_line    0x00000928       0x90 Objects - Graphics Primitives Layer Demo\GroupBox.o
 .debug_line    0x000009b8       0x90 Objects - Graphics Primitives Layer Demo\ListBox.o
 .debug_line    0x00000a48       0x90 Objects - Graphics Primitives Layer Demo\Meter.o
 .debug_line    0x00000ad8       0x90 Objects - Graphics Primitives Layer Demo\Picture.o
 .debug_line    0x00000b68      0x416 Objects - Graphics Primitives Layer Demo\Primitive.o
 .debug_line    0x00000f7e       0x90 Objects - Graphics Primitives Layer Demo\ProgressBar.o
 .debug_line    0x0000100e       0x90 Objects - Graphics Primitives Layer Demo\RadioButton.o
 .debug_line    0x0000109e       0x90 Objects - Graphics Primitives Layer Demo\RoundDial.o
 .debug_line    0x0000112e       0x90 Objects - Graphics Primitives Layer Demo\Slider.o
 .debug_line    0x000011be       0x90 Objects - Graphics Primitives Layer Demo\StaticText.o
 .debug_line    0x0000124e      0x480 Objects - Graphics Primitives Layer Demo\DisplayDriver.o
 .debug_line    0x000016ce       0xeb C:/Program Files/Microchip/MPLAB C32/bin/../lib/gcc/pic32mx/3.4.4/../../../../pic32mx/lib/size\libc.a(memcpy.o)
 .debug_line    0x000017b9       0xcd C:/Program Files/Microchip/MPLAB C32/bin/../lib/gcc/pic32mx/3.4.4/../../../../pic32mx/lib/size\libc.a(general-exception.o)
 .debug_line    0x00001886       0x7a C:/Program Files/Microchip/MPLAB C32/bin/../lib/gcc/pic32mx/3.4.4/../../../../pic32mx/lib/size\libc.a(exit.o)
 .debug_line    0x00001900       0x81 C:/Program Files/Microchip/MPLAB C32/bin/../lib/gcc/pic32mx/3.4.4/../../../../pic32mx/lib/size\libc.a(_iobfuncs.o)
 .debug_line    0x00001981       0x7d C:/Program Files/Microchip/MPLAB C32/bin/../lib/gcc/pic32mx/3.4.4/../../../../pic32mx/lib/size\libc.a(stubs.o)
 .debug_line    0x000019fe       0x99 C:/Program Files/Microchip/MPLAB C32/bin/../lib/gcc/pic32mx/3.4.4/../../../../pic32mx/lib/size\libc.a(default-general-exception-handler.o)
 .debug_line    0x00001a97       0x9b C:/Program Files/Microchip/MPLAB C32/bin/../lib/gcc/pic32mx/3.4.4/../../../../pic32mx/lib/size\libc.a(default-bootstrap-exception-handler.o)
 .debug_line    0x00001b32       0x88 C:/Program Files/Microchip/MPLAB C32/bin/../lib/gcc/pic32mx/3.4.4/../../../../pic32mx/lib/size\libc.a(default-on-reset.o)
 .debug_line    0x00001bba       0x8c C:/Program Files/Microchip/MPLAB C32/bin/../lib/gcc/pic32mx/3.4.4/../../../../pic32mx/lib/size\libc.a(default-on-bootstrap.o)
 .debug_line    0x00001c46       0x9f C:/Program Files/Microchip/MPLAB C32/bin/../lib/gcc/pic32mx/3.4.4/../../../../pic32mx/lib/size\libc.a(default-nmi-handler.o)
 .debug_line    0x00001ce5       0x81 C:/Program Files/Microchip/MPLAB C32/bin/../lib/gcc/pic32mx/3.4.4/../../../../pic32mx/lib/size\libc.a(_mon_getc.o)
 .debug_line    0x00001d66       0x82 C:/Program Files/Microchip/MPLAB C32/bin/../lib/gcc/pic32mx/3.4.4/../../../../pic32mx/lib/size\libc.a(_mon_write.o)
 .debug_line    0x00001de8       0x7d C:/Program Files/Microchip/MPLAB C32/bin/../lib/gcc/pic32mx/3.4.4/../../../../pic32mx/lib/size\libc.a(_exit.o)
 .debug_line    0x00001e65       0x81 C:/Program Files/Microchip/MPLAB C32/bin/../lib/gcc/pic32mx/3.4.4/../../../../pic32mx/lib/size\libc.a(_mon_putc.o)
 .debug_line    0x00001ee6       0xa0 C:/Program Files/Microchip/MPLAB C32/bin/../lib/gcc/pic32mx/3.4.4/../../../../pic32mx/lib/size\libmchp_peripheral.a(int_disable_interrupts_lib.o)
 .debug_line    0x00001f86       0x9b C:/Program Files/Microchip/MPLAB C32/bin/../lib/gcc/pic32mx/3.4.4/../../../../pic32mx/lib/size\libmchp_peripheral.a(int_enable_mv_int_lib.o)
 .debug_line    0x00002021       0xa0 C:/Program Files/Microchip/MPLAB C32/bin/../lib/gcc/pic32mx/3.4.4/../../../../pic32mx/lib/size\libmchp_peripheral.a(int_restore_interrupts_lib.o)
 .debug_line    0x000020c1       0x9b C:/Program Files/Microchip/MPLAB C32/bin/../lib/gcc/pic32mx/3.4.4/../../../../pic32mx/lib/size\libmchp_peripheral.a(open_core_timer_lib.o)
 .debug_line    0x0000215c       0x8f C:/Program Files/Microchip/MPLAB C32/bin/../lib/gcc/pic32mx/3.4.4/../../../../pic32mx/lib/size\libmchp_peripheral.a(pcache.o)
 .debug_line    0x000021eb       0x9f C:/Program Files/Microchip/MPLAB C32/bin/../lib/gcc/pic32mx/3.4.4/../../../../pic32mx/lib/size\libmchp_peripheral.a(int_enable_interrupts_lib.o)

.debug_frame    0x00000000      0x9a8
 *(.debug_frame)
 .debug_frame   0x00000000       0x44 Objects - Graphics Primitives Layer Demo\MainDemo.o
 .debug_frame   0x00000044      0x1c8 Objects - Graphics Primitives Layer Demo\Primitive.o
 .debug_frame   0x0000020c      0x370 Objects - Graphics Primitives Layer Demo\DisplayDriver.o
 .debug_frame   0x0000057c       0x34 C:/Program Files/Microchip/MPLAB C32/bin/../lib/gcc/pic32mx/3.4.4/../../../../pic32mx/lib/size\libc.a(exit.o)
 .debug_frame   0x000005b0       0x98 C:/Program Files/Microchip/MPLAB C32/bin/../lib/gcc/pic32mx/3.4.4/../../../../pic32mx/lib/size\libc.a(_iobfuncs.o)
 .debug_frame   0x00000648      0x178 C:/Program Files/Microchip/MPLAB C32/bin/../lib/gcc/pic32mx/3.4.4/../../../../pic32mx/lib/size\libc.a(stubs.o)
 .debug_frame   0x000007c0       0x20 C:/Program Files/Microchip/MPLAB C32/bin/../lib/gcc/pic32mx/3.4.4/../../../../pic32mx/lib/size\libc.a(default-general-exception-handler.o)
 .debug_frame   0x000007e0       0x20 C:/Program Files/Microchip/MPLAB C32/bin/../lib/gcc/pic32mx/3.4.4/../../../../pic32mx/lib/size\libc.a(default-bootstrap-exception-handler.o)
 .debug_frame   0x00000800       0x20 C:/Program Files/Microchip/MPLAB C32/bin/../lib/gcc/pic32mx/3.4.4/../../../../pic32mx/lib/size\libc.a(default-on-reset.o)
 .debug_frame   0x00000820       0x20 C:/Program Files/Microchip/MPLAB C32/bin/../lib/gcc/pic32mx/3.4.4/../../../../pic32mx/lib/size\libc.a(default-on-bootstrap.o)
 .debug_frame   0x00000840       0x20 C:/Program Files/Microchip/MPLAB C32/bin/../lib/gcc/pic32mx/3.4.4/../../../../pic32mx/lib/size\libc.a(_mon_getc.o)
 .debug_frame   0x00000860       0x30 C:/Program Files/Microchip/MPLAB C32/bin/../lib/gcc/pic32mx/3.4.4/../../../../pic32mx/lib/size\libc.a(_mon_write.o)
 .debug_frame   0x00000890       0x20 C:/Program Files/Microchip/MPLAB C32/bin/../lib/gcc/pic32mx/3.4.4/../../../../pic32mx/lib/size\libc.a(_exit.o)
 .debug_frame   0x000008b0       0x20 C:/Program Files/Microchip/MPLAB C32/bin/../lib/gcc/pic32mx/3.4.4/../../../../pic32mx/lib/size\libc.a(_mon_putc.o)
 .debug_frame   0x000008d0       0x20 C:/Program Files/Microchip/MPLAB C32/bin/../lib/gcc/pic32mx/3.4.4/../../../../pic32mx/lib/size\libmchp_peripheral.a(int_disable_interrupts_lib.o)
 .debug_frame   0x000008f0       0x28 C:/Program Files/Microchip/MPLAB C32/bin/../lib/gcc/pic32mx/3.4.4/../../../../pic32mx/lib/size\libmchp_peripheral.a(int_enable_mv_int_lib.o)
 .debug_frame   0x00000918       0x20 C:/Program Files/Microchip/MPLAB C32/bin/../lib/gcc/pic32mx/3.4.4/../../../../pic32mx/lib/size\libmchp_peripheral.a(int_restore_interrupts_lib.o)
 .debug_frame   0x00000938       0x20 C:/Program Files/Microchip/MPLAB C32/bin/../lib/gcc/pic32mx/3.4.4/../../../../pic32mx/lib/size\libmchp_peripheral.a(open_core_timer_lib.o)
 .debug_frame   0x00000958       0x30 C:/Program Files/Microchip/MPLAB C32/bin/../lib/gcc/pic32mx/3.4.4/../../../../pic32mx/lib/size\libmchp_peripheral.a(pcache.o)
 .debug_frame   0x00000988       0x20 C:/Program Files/Microchip/MPLAB C32/bin/../lib/gcc/pic32mx/3.4.4/../../../../pic32mx/lib/size\libmchp_peripheral.a(int_enable_interrupts_lib.o)

.debug_str      0x00000000     0x185f
 *(.debug_str)
 .debug_str     0x00000000      0x305 Objects - Graphics Primitives Layer Demo\MainDemo.o
                                0x357 (size before relaxing)
 .debug_str     0x00000305       0x6c Objects - Graphics Primitives Layer Demo\Pictures PIC32.o
                                0x2b2 (size before relaxing)
 .debug_str     0x00000371       0x15 Objects - Graphics Primitives Layer Demo\Font25PixelsHeight.o
                                 0x9d (size before relaxing)
 .debug_str     0x00000386       0x1f Objects - Graphics Primitives Layer Demo\Window.o
                                0x234 (size before relaxing)
 .debug_str     0x000003a5       0x1f Objects - Graphics Primitives Layer Demo\Button.o
                                0x234 (size before relaxing)
 .debug_str     0x000003c4       0x1e Objects - Graphics Primitives Layer Demo\Chart.o
                                0x233 (size before relaxing)
 .debug_str     0x000003e2       0x21 Objects - Graphics Primitives Layer Demo\CheckBox.o
                                0x236 (size before relaxing)
 .debug_str     0x00000403       0x20 Objects - Graphics Primitives Layer Demo\EditBox.o
                                0x235 (size before relaxing)
 .debug_str     0x00000423       0x1c Objects - Graphics Primitives Layer Demo\GOL.o
                                0x231 (size before relaxing)
 .debug_str     0x0000043f       0x1d Objects - Graphics Primitives Layer Demo\Grid.o
                                0x232 (size before relaxing)
 .debug_str     0x0000045c       0x21 Objects - Graphics Primitives Layer Demo\GroupBox.o
                                0x236 (size before relaxing)
 .debug_str     0x0000047d       0x20 Objects - Graphics Primitives Layer Demo\ListBox.o
                                0x235 (size before relaxing)
 .debug_str     0x0000049d       0x1e Objects - Graphics Primitives Layer Demo\Meter.o
                                0x233 (size before relaxing)
 .debug_str     0x000004bb       0x20 Objects - Graphics Primitives Layer Demo\Picture.o
                                0x235 (size before relaxing)
 .debug_str     0x000004db      0x3ce Objects - Graphics Primitives Layer Demo\Primitive.o
                                0x663 (size before relaxing)
 .debug_str     0x000008a9       0x24 Objects - Graphics Primitives Layer Demo\ProgressBar.o
                                0x239 (size before relaxing)
 .debug_str     0x000008cd       0x24 Objects - Graphics Primitives Layer Demo\RadioButton.o
                                0x239 (size before relaxing)
 .debug_str     0x000008f1       0x22 Objects - Graphics Primitives Layer Demo\RoundDial.o
                                0x237 (size before relaxing)
 .debug_str     0x00000913       0x1f Objects - Graphics Primitives Layer Demo\Slider.o
                                0x234 (size before relaxing)
 .debug_str     0x00000932       0x23 Objects - Graphics Primitives Layer Demo\StaticText.o
                                0x238 (size before relaxing)
 .debug_str     0x00000955      0x3d6 Objects - Graphics Primitives Layer Demo\DisplayDriver.o
                                0x685 (size before relaxing)
 .debug_str     0x00000d2b       0x5d C:/Program Files/Microchip/MPLAB C32/bin/../lib/gcc/pic32mx/3.4.4/../../../../pic32mx/lib/size\libc.a(exit.o)
                                 0x89 (size before relaxing)
 .debug_str     0x00000d88       0xae C:/Program Files/Microchip/MPLAB C32/bin/../lib/gcc/pic32mx/3.4.4/../../../../pic32mx/lib/size\libc.a(_iobfuncs.o)
                                 0xd5 (size before relaxing)
 .debug_str     0x00000e36      0x2d0 C:/Program Files/Microchip/MPLAB C32/bin/../lib/gcc/pic32mx/3.4.4/../../../../pic32mx/lib/size\libc.a(stubs.o)
                                0x2f7 (size before relaxing)
 .debug_str     0x00001106       0x97 C:/Program Files/Microchip/MPLAB C32/bin/../lib/gcc/pic32mx/3.4.4/../../../../pic32mx/lib/size\libc.a(default-general-exception-handler.o)
                                 0xbe (size before relaxing)
 .debug_str     0x0000119d       0x9b C:/Program Files/Microchip/MPLAB C32/bin/../lib/gcc/pic32mx/3.4.4/../../../../pic32mx/lib/size\libc.a(default-bootstrap-exception-handler.o)
                                 0xc2 (size before relaxing)
 .debug_str     0x00001238       0x75 C:/Program Files/Microchip/MPLAB C32/bin/../lib/gcc/pic32mx/3.4.4/../../../../pic32mx/lib/size\libc.a(default-on-reset.o)
                                 0x9c (size before relaxing)
 .debug_str     0x000012ad       0x7d C:/Program Files/Microchip/MPLAB C32/bin/../lib/gcc/pic32mx/3.4.4/../../../../pic32mx/lib/size\libc.a(default-on-bootstrap.o)
                                 0xa4 (size before relaxing)
 .debug_str     0x0000132a       0x6e C:/Program Files/Microchip/MPLAB C32/bin/../lib/gcc/pic32mx/3.4.4/../../../../pic32mx/lib/size\libc.a(_mon_getc.o)
                                 0x95 (size before relaxing)
 .debug_str     0x00001398       0x70 C:/Program Files/Microchip/MPLAB C32/bin/../lib/gcc/pic32mx/3.4.4/../../../../pic32mx/lib/size\libc.a(_mon_write.o)
                                 0x97 (size before relaxing)
 .debug_str     0x00001408       0x66 C:/Program Files/Microchip/MPLAB C32/bin/../lib/gcc/pic32mx/3.4.4/../../../../pic32mx/lib/size\libc.a(_exit.o)
                                 0x8d (size before relaxing)
 .debug_str     0x0000146e       0x6e C:/Program Files/Microchip/MPLAB C32/bin/../lib/gcc/pic32mx/3.4.4/../../../../pic32mx/lib/size\libc.a(_mon_putc.o)
                                 0x95 (size before relaxing)
 .debug_str     0x000014dc       0x98 C:/Program Files/Microchip/MPLAB C32/bin/../lib/gcc/pic32mx/3.4.4/../../../../pic32mx/lib/size\libmchp_peripheral.a(int_disable_interrupts_lib.o)
                                 0xbf (size before relaxing)
 .debug_str     0x00001574       0x9e C:/Program Files/Microchip/MPLAB C32/bin/../lib/gcc/pic32mx/3.4.4/../../../../pic32mx/lib/size\libmchp_peripheral.a(int_enable_mv_int_lib.o)
                                 0xc5 (size before relaxing)
 .debug_str     0x00001612       0x98 C:/Program Files/Microchip/MPLAB C32/bin/../lib/gcc/pic32mx/3.4.4/../../../../pic32mx/lib/size\libmchp_peripheral.a(int_restore_interrupts_lib.o)
                                 0xbf (size before relaxing)
 .debug_str     0x000016aa       0x8c C:/Program Files/Microchip/MPLAB C32/bin/../lib/gcc/pic32mx/3.4.4/../../../../pic32mx/lib/size\libmchp_peripheral.a(open_core_timer_lib.o)
                                 0xb3 (size before relaxing)
 .debug_str     0x00001736       0x93 C:/Program Files/Microchip/MPLAB C32/bin/../lib/gcc/pic32mx/3.4.4/../../../../pic32mx/lib/size\libmchp_peripheral.a(pcache.o)
                                 0xba (size before relaxing)
 .debug_str     0x000017c9       0x96 C:/Program Files/Microchip/MPLAB C32/bin/../lib/gcc/pic32mx/3.4.4/../../../../pic32mx/lib/size\libmchp_peripheral.a(int_enable_interrupts_lib.o)
                                 0xbd (size before relaxing)

.debug_loc
 *(.debug_loc)

.debug_macinfo
 *(.debug_macinfo)

.debug_weaknames
 *(.debug_weaknames)

.debug_funcnames
 *(.debug_funcnames)

.debug_typenames
 *(.debug_typenames)

.debug_varnames
 *(.debug_varnames)

/DISCARD/
 *(.note.GNU-stack)
OUTPUT(Objects - Graphics Primitives Layer Demo\Primitives Layer Demo PIC32.elf elf32-tradlittlemips)

.mdebug.abi32   0x9d07e148        0x0

.debug_ranges   0x9d07e148       0x18
 .debug_ranges  0x9d07e148       0x18 Objects - Graphics Primitives Layer Demo\MainDemo.o

.rel.dyn        0x9d07e160        0x0
